:020000040000fa
:080000000002040000000000f2
:020000040000fa
:100400002f622100007f240000018800000000000e
:100410000a00070011000700000020000000e000b3
:10042000020032000000020000000000ca4002008a
:10043000000000000040da000000fe004440a90077
:1004400080c121000000e000030032000000200015
:10045000a00188004440a800000006006034250088
:10046000010020001500370062004000e0804800d5
:10047000910188009001ba0062004000e0804800cd
:10048000910188009002ba0062004000e0804800bc
:100490000002eb006028e10004003a000059eb0084
:1004a0008301e900fdff3e00040037006128e10000
:1004b000010032000082eb00050007009101880076
:1004c0001001ba000200e000e7ff3a00000005005a
:1004d000910188008002780062004000e0804800be
:1004e0003559ba008301e900080032002559ba00e5
:1004f0008301e900050032000400e000f4ff32004f
:1005000015d9ba008301e900f1ff3a0000000600a6
:100510008001eb0002003700817178008301e80060
:10052000828f5100fcff3a0000000600889fbe0049
:100530008a9fbe008c1f78005c01070063013300b6
:1005400003866c006450e1002e0032006420e1005c
:10055000330032006150e1002f0032006120e100e1
:100560003100320085855500eb07b00009002000fe
:1005700008042000050037000804440089844c006a
:100580000a0031000603430087834b00000153003b
:1005900081815b00f8ff33000203be000800a00069
:1005a0000804440089844c00f6ff3900c639dd0098
:1005b0008301730001003200130020008904d10080
:1005c0000884d3000998a300050032000800a700a2
:1005d0000300a0008904d1000884d3008b05e80043
:1005e0008904d1000884d3000001eb000281d2000d
:1005f0004601070001f0a1000cf0a70001f0a000e7
:100600003b0137006420e1003d0132000801be00db
:100610000200be00f7ff37006120e1003801320020
:100620006000b800f3ff37000000200001f8270049
:10063000f0ff3700889fbe008a9fbe008c1f7800a5
:100640001a0107002101330003866c006450e100a9
:10065000240032006420e100270032006150e100f4
:10066000220032006120e100210032008b8542002f
:10067000eb07b1000134b800003ab80008044200aa
:1006800089844a00013ab8000030b80088804000f0
:1006900009014a0004003300000040008180480046
:1006a000020149008b05e900c909dd0083017000e2
:1006b0000100320013002000c814de004814dd00e1
:1006c0004709de001200b200c808de00088470008e
:1006d0000e01070001f0a1000cf0a70001f0a0003e
:1006e000030137006120e100050132000801be006e
:1006f0000200be00f7ff37006150e100fcff3a0046
:10070000ff0037000081eb00260137000001eb00fd
:1007100024013700f4ff2f008b01370003f0a20003
:10072000889fbe008a9fbe008c1f7800df000700f4
:10073000e60033006450e1004f0032006420e10025
:100740005200320003826c0007003b000905d00014
:100750000306d000820f54000c065d000200390031
:100760000200320089017800030678008582550076
:1007700004003d000003fd008103fd008502ea0046
:100780008b854200840f720002003b006000100065
:10079000e08018006011b8000005eb007a28e10045
:1007a0000a00390006007800c75ddd00f707b200d7
:1007b000878075002d003700828171000a01780062
:1007c000610560008180d1000080d3008502e900ce
:1007d000f9ff3b00060440008784480002003b000c
:1007e00060041400e0841c000988a30007003200a4
:1007f0008a81710082817100610164008904d100e5
:100800000884d3008b05e800170037000978a3009f
:1008100013003a000b00e000130034008b05e900e0
:100820000804440089844c000a4474000978a30039
:100830000d003a000b00e000070034008b05e900d2
:100840000804440089844c0001003a000b00200099
:100850000978a300f7ff32000001eb000200370027
:10086000828171000a017800a80007000cf0a7003f
:1008700001f0a0009e0037006420e10002003a0071
:10088000838f6c009e0033000801be000200be0092
:10089000970037000001be00460107000470a70062
:1008a00003f0a1006509b100160032000d0035000b
:1008b0006828e10006003500f0ff2f00f1ff270057
:1008c0000300e00013003b000100280000000500c9
:1008d00000004000818048008502e900fcff3a00ea
:1008e00008003700f88f420002003c008000eb0057
:1008f000000005008100d1000080d3008502e800df
:10090000fcff3a000300e00002003b006000100022
:10091000e080180000000600889fbe008a9fbe008d
:10092000010578000100e0000400350008003c00eb
:100930000000e000200032000500370060001000d9
:10094000e080180002003b0001f02c001a00370084
:100950000004be006011b8006b0920000982cf00be
:10096000020039000882cf000441b0006942520001
:100970000e00320008003b008281710061016400ba
:100980008904d1000884d3008b05e8000442e80004
:10099000f9ff3a00050037000804440089844c0040
:1009a0008b05e9000442e900fbff3a00570007000d
:1009b0000af0a70001f0a0004f05be004f04be00e2
:1009c00000000600839f68000100e00002003d0077
:1009d00060001000e08018000300e00002003d000d
:1009e00060011100e0811900050007004f00e000e0
:1009f00002003b0060001000e080180000000600cc
:100a00006022b800060220000000d0008180d200e1
:100a10000482d2008582d2000000a00002025200af
:100a200083825a00030031000202420083824a009e
:100a30000000a1000603e900f3ff3a0000000600f1
:100a40000001be00db0007000470a70003f0a10056
:100a500003f8a30013003a006509b100100032004a
:100a6000090035006928e100020035000100280076
:100a70000000050000004000818048008502e90078
:100a8000fcff3a0000000600f88f42000500350028
:100a90008100d1000080d3008502e800fcff3a000d
:100aa000000006008000eb00000005000004be000e
:100ab000c00007000003be000405be000200be0027
:100ac000bc000700844f7500000006000200be0055
:100ad0006450e100050036006420e10002003600a9
:100ae0000968a30001003a000800be000160a000f0
:100af0004f0678004f05be004f04be000000060000
:100b0000f0ff2f00f1ff2700f9ff370081002000e0
:100b1000618055000b003d000b00200061fe2f009e
:100b20000100e1001d003400828171006101640058
:100b30008904d1000884d3000000e800faff3a00dd
:100b4000710020006100640003007000020060007a
:100b50000900320061044400e0844c000988a500cb
:100b6000050032008b05e8006808e10002003a0049
:100b70008904d1000884d300f20f20000258e1005c
:100b800005003d00c75ddd00f907b20089807500f2
:100b900008007800000006000bf827008b007800a2
:100ba00000000500889fbe008a9fbe008c9fbe008b
:100bb000820578000004be007e0007000800be0029
:100bc0006420e1000700390002003a00f1ff27002d
:100bd000f0ff2f000160a0001202200002a1880097
:100be000550037006120e10003003a000b00a70028
:100bf00001f823005000370001f0a100020021009d
:100c000093642400800007000800be000400350043
:100c1000b2fd2000930c24007d0007000004be00fc
:100c20000005eb000b00a6004f0dde0001f0a10057
:100c30000004be0032982f0023ea23007dfe070047
:100c40000001eb0003f023000b00a70003f82300d2
:100c5000b3fe07000fff07000000a7000a00a20074
:100c60002dff07000b00e00003003200020020000f
:100c700003f02300a9fe070001f0a2000006be0059
:100c800002002000930424006afe07000801be0051
:100c9000a3fe0700809fbe000c00be0022a22a0017
:100ca000d3a7230063fe07004f01be009cfe070090
:100cb0000004be0001f0a100020020000398230000
:100cc000510007000800be00190035000001be00f9
:100cd00058fe07000006be00b2c52900e3622300eb
:100ce00054fe070022222b00f3942b008cfe0700f9
:100cf0000c01be004ffe0700e273280083c02300f2
:100d000087fe07000c01be004afe070042aa2a0027
:100d1000a3e22b0082fe07000c01be0045fe070087
:100d20000801be0043fe07000801be007cfe07006c
:100d30000a00a70001f0a2004f06be004f05be004a
:100d40004f04be0000000600889fbe008a9fbe00c0
:100d5000841f780055ff07004f0078001100330012
:100d6000f0ff2f00838f6c0006003b000405650038
:100d70000a00a7000800370009f0a60010002000b4
:100d800008003700820f5400838f5c000300390095
:100d90001000200001003e000000200009f0a70024
:100da0000000ea004f05be004f04be000000e00056
:100db00000000600c70ade00f107b200f50fb2001e
:100dc00008003200e1cf4200020032000170a000b2
:100dd00024000500810f70000100320004080500a6
:100de00044000500810f700002003a001400050065
:100df0008502e9000000400081c04800fcff3b0084
:100e00000170a0002400050014002000ceff370070
:100e10000400200000003700889fbe008a9fbe00ab
:100e20008c1f78004f26dd0020ff070027ff3300ce
:100e30006120e100430032006250e10041003e00c9
:100e40003e0039006420e1003c003200058255007c
:100e50000f003b000402e80038003a00800f530006
:100e6000818f5b00350034000800be0003f0a10054
:100e700001f0a60003f0a0000cf0a70028fe070078
:100e80001bff37000603430087834b000c464600d8
:100e90000005530081855b00020033000a03be0099
:100ea0000c00a0000402e900f6ff3b008505780075
:100eb0000602430087824b0004003a006000b8003d
:100ec00009f0a70001f0a00009ff3700000252005e
:100ed00081825a000704e000040033000603430047
:100ee00087834b008b05e900faff3700090578007e
:100ef0000604be000203be006011b80003ff070035
:100f0000e00f5200e08f5a000700350002003c005d
:100f10000c08a300040032000601be0003f0a0008c
:100f20000cf0a700fefd07000a85680001f0a10093
:100f30000af0a70001f0a000edfe37000800be0097
:100f4000ebfe3700100220000cf0a60000a1880084
:100f5000ebfe370023c2bf000004a2006100600066
:100f60000000060033c2bf000004a2006100600060
:100f70000000060021e2a9009560a9009580a90063
:100f80008560a9008580a9000000060031e2a90063
:100f900097c0a90097e0a90087c0a90087e0a90031
:100fa000000006008560a9008580a900e741600077
:100fb000c419dd00910a200091407800f2c8b30006
:100fc00082c0600083c070008000fd00a9e0b7000f
:100fd0008000fd00800178000307b200c419de0024
:100fe000a10a20009140780082cfb30082c0600047
:100ff00083c070008000fd00aae0b7008000fd0003
:10100000680160004311de004311dd00510920003a
:10101000914078000134a10082c070008000fd0082
:1010200095e0b7008000fd000008b2004700de0038
:101030004400dd0051092000914078000144a100e6
:1010400080c070000100780095e0b7000000060045
:1010500087c0a90087e0a900e7416000310b2000ac
:101060009140780082cfb30082c0600083c07000de
:101070008000fd00b3e0b7008000fd0001c7b300b1
:1010800081416000310b200091407800f2c8b3002c
:1010900082c0600083c070008000fd00b3e0b70034
:1010a0008000fd00680160004311de004611dd0094
:1010b00071092000914078000164a10082c0700095
:1010c0008000fd0097e0b7008000fd000008b2003e
:1010d0004700de00614060004700dd00710920002c
:1010e000914078000174a10080c070000100780078
:1010f00097e0b7000000060022c2bf006100600058
:101100000000060032c2bf0061006000000006005f
:10111000889fbe008a9fbe008c9fbe008e1f7800f5
:101120000005780001067800820478000107780045
:101130008006eb000000e00013003a0015003700c5
:10114000890f5400140031000804e800eaff07008a
:101150000004e000faff320020c2bf0066406000d9
:10116000e64f500003003a0030118000001e780066
:101170000200370030118000005f78008d06e80023
:101180008a8f5600030032008d0555000004eb00e5
:10119000eeff37008005eb000b0078004f0778006a
:1011a0004f06be004f05be004f04be000000060003
:1011b000889fbe008a9fbe008c9fbe008e1f780055
:1011c00000057800010678008204780001077800a5
:1011d0008006eb000000e00013003a001500370025
:1011e000890f5400140031000804e800c5ff07000f
:1011f0000004e000faff320030c2bf006640600029
:10120000e64f500003003a00b0118000001e780045
:1012100002003700b0118000005f78008d06e80002
:101220008a8f5600030032008d0555000004eb0044
:10123000eeff37008005eb000b0078004f077800c9
:101240004f06be004f05be004f04be000000060062
:10125000421188000011880011118800000006006a
:10126000c2118800801188009111880000000600da
:10127000000178008000780023c2bf000018a3009e
:10128000fdff3a0020c2bf0066406000e64f5000fc
:1012900010003a0005003700201188000281e800a4
:1012a00023c2bf000018a300fdff3a00120078001f
:1012b0000000e000f8ff3a00090037000000fb00e2
:1012c000201188008100e80023c2bf000018a3009d
:1012d000fdff3a00114078000004e000f7ff3a00fb
:1012e00000000600000178008000780033c2bf00d3
:1012f0000018a300fdff3a0030c2bf006640600046
:10130000e64f500010003a0005003700a011880099
:101310000281e80033c2bf000018a300fdff3a00bd
:10132000120078000000e000f8ff3a0009003700e2
:101330000000fb00a01188008100e80033c2bf005c
:101340000018a300fdff3a00114078000004e000ff
:10135000f7ff3a000000060020c2bf0066406000b0
:10136000e64f500002003a003011800002003700c2
:10137000301180000080fb000000060030c2bf007a
:1013800066406000e64f500002003a00b011800055
:1013900002003700b01180000080fb000000060052
:1013a0008000780023c2bf000018a300fdff3a00b0
:1013b00020c2bf0066406000e64f500002003a00c5
:1013c00021118800020037000180fb0020118800f5
:1013d000000006008000780033c2bf000018a300a0
:1013e000fdff3a0030c2bf0066406000e64f50008b
:1013f00002003a00a1118800020037000180fb00c2
:08140000a011880000000600a5
:020000040000fa
:0200000401f009
:04000000ffff0000fe
:020000040000fa
:0200000401f009
:04000400ffff0000fa
:020000040000fa
:0200000401f009
:04000c00faff0000f7
:020000040000fa
:0200000401f009
:040010007eff00006f
:020000040000fa
:0200000401f009
:040014007fff00006a
:020000040000fa
:0200000401f009
:04001800feff0000e7
:020000040000fa
:10000800f2590000de450000f045000002460000fd
:1000180014460000f2590000f2590000f25900009d
:10002800f2590000f2590000f2590000484500005a
:10003800f2590000f2590000f2590000f25900008c
:100048002e590000f2590000f259000082450000c4
:1000580054450000f2590000f2590000f25900001e
:10006800aa540000f2590000f2590000f2590000a9
:10007800f2590000f2590000f2590000f25900004c
:10008800f2590000f2590000f2590000f25900003c
:10009800f2590000f2590000da450000d645000088
:1000a800f2590000f2590000f2590000f25900001c
:1000b800f2590000f2590000f2590000f45800000b
:1000c800f2590000f2590000f2590000f2590000fc
:1000d800f2590000f2590000f2590000f2590000ec
:1000e800f2590000f25900001a4d0000f2590000c0
:1000f800f2590000f2590000f2590000f2590000cc
:10010800f2590000f2590000f2590000f2590000bb
:10011800f2590000f2590000f2590000f2590000ab
:10012800f2590000f2590000f2590000f25900009b
:10013800f2590000f2590000f2590000f25900008b
:10014800f2590000f2590000f2590000f25900007b
:10015800f2590000f2590000f2590000f25900006b
:10016800f2590000f2590000f2590000f25900005b
:10017800f2590000f2590000f2590000f25900004b
:10018800f2590000f2590000f2590000f25900003b
:10019800f2590000f2590000f2590000f25900002b
:1001a800f2590000f2590000f2590000f25900001b
:1001b800f2590000f2590000f2590000f25900000b
:1001c800f2590000f2590000f2590000f2590000fb
:1001d800f2590000f2590000f2590000f2590000eb
:1001e800f2590000f2590000f2590000f2590000db
:0801f800f2590000f259000069
:020000040000fa
:10020800f2590000de450000f045000002460000fb
:1002180014460000f2590000f2590000f25900009b
:10022800f2590000f2590000f25900004845000058
:10023800f2590000f2590000f2590000f25900008a
:100248002e590000f2590000f259000082450000c2
:1002580054450000f2590000f2590000f25900001c
:10026800aa540000f2590000f2590000f2590000a7
:10027800f2590000f2590000f2590000f25900004a
:10028800f2590000f2590000f2590000f25900003a
:10029800f2590000f2590000da450000d645000086
:1002a800f2590000f2590000f2590000f25900001a
:1002b800f2590000f2590000f2590000f458000009
:1002c800f2590000f2590000f2590000f2590000fa
:1002d800f2590000f2590000f2590000f2590000ea
:1002e800f2590000f25900001a4d0000f2590000be
:1002f800f2590000f2590000f2590000f2590000ca
:10030800f2590000f2590000f2590000f2590000b9
:10031800f2590000f2590000f2590000f2590000a9
:10032800f2590000f2590000f2590000f259000099
:10033800f2590000f2590000f2590000f259000089
:10034800f2590000f2590000f2590000f259000079
:10035800f2590000f2590000f2590000f259000069
:10036800f2590000f2590000f2590000f259000059
:10037800f2590000f2590000f2590000f259000049
:10038800f2590000f2590000f2590000f259000039
:10039800f2590000f2590000f2590000f259000029
:1003a800f2590000f2590000f2590000f259000019
:1003b800f2590000f2590000f2590000f259000009
:1003c800f2590000f2590000f2590000f2590000f9
:1003d800f2590000f2590000f2590000f2590000e9
:1003e800f2590000f2590000f2590000f2590000d9
:0803f800f2590000f259000067
:020000040000fa
:1014080000000000cd0100008c0200001f03000056
:101418009b030000080400006b040000c6040000e1
:101428001b0500006b050000b6050000fe05000066
:101438004306000085060000c506000002070000fc
:101448003e07000077070000af070000e60700002e
:101458001b0800004f08000082080000b4080000c4
:10146800e4080000140900004309000071090000a5
:101478009e090000ca090000f6090000210a0000c0
:101488004b0a0000750a00009e0a0000c70a000007
:10149800ef0a0000170b00003e0b0000640b000071
:1014a8008b0b0000b00b0000d60b0000fb0b0000fc
:1014b8001f0c0000430c0000670c00008b0c0000a0
:1014c800ae0c0000d00c0000f30c0000150d00005d
:1014d800370d0000590d00007a0d00009b0d00002b
:1014e800bc0d0000dc0d0000fc0d00001c0e00000f
:1014f8003c0e00005c0e00007b0e00009a0e0000ff
:10150800b90e0000d80e0000f60e0000150f0000fe
:10151800330f0000510f00006e0f00008c0f000009
:10152800a90f0000c60f0000e40f00000010000023
:101538001d1000003a100000561000007210000044
:101548008f100000ab100000c6100000e210000071
:10155800fe100000191100003411000050110000a5
:101568006b11000086110000a0110000bb110000e3
:10157800d6110000f01100000b1200002512000027
:101588003f12000059120000731200008d12000073
:10159800a6120000c0120000da120000f3120000c8
:1015a8000c130000261300003f130000581300001e
:1015b800711300008a130000a3130000bc1300007d
:1015c800d4130000ed130000051400001e140000e1
:1015d800361400004e140000671400007f14000049
:1015e80097140000af140000c7140000df140000b7
:1015f800f71400000e150000261500003e15000027
:10160800551500006d150000841500009b1500009d
:10161800b3150000ca150000e1150000f815000018
:101628000f160000271600003d1600005416000093
:101638006b1600008216000099160000b016000014
:10164800c6160000dd160000f41600000a17000098
:1016580021170000371700004d170000641700001d
:101668007a17000090170000a7170000bd170000a8
:10167800d3170000e9170000ff1700001518000035
:101688002b18000041180000571800006d180000c2
:101698008318000099180000ae180000c418000054
:1016a800da180000ef180000051900001b190000e7
:1016b80030190000461900005b190000711900007c
:1016c800861900009c190000b1190000c619000015
:1016d800dc190000f1190000061a00001c1a0000ad
:1016e800311a0000461a00005b1a0000711a000047
:1016f800861a00009b1a0000b01a0000c51a0000e4
:10170800da1a0000ef1a0000041b0000191b000081
:101718002e1b0000431b0000581b00006d1b00001f
:10172800821b0000971b0000ab1b0000c01b0000c1
:10173800d51b0000ea1b0000ff1b0000131c000063
:10174800281c00003d1c0000521c0000661c000004
:101758007b1c0000901c0000a41c0000b91c0000a9
:10176800ce1c0000e21c0000f71c00000b1d00004e
:10177800201d0000351d0000491d00005e1d0000f1
:10178800721d0000871d00009b1d0000b01d000099
:10179800c41d0000d91d0000ed1d0000021e000040
:1017a800161e00002b1e00003f1e0000531e0000e6
:1017b800681e00007c1e0000911e0000a51e00008f
:1017c800ba1e0000ce1e0000e21e0000f71e000038
:1017d8000b1f0000201f0000341f0000481f0000de
:1017e8005d1f0000711f0000861f00009a1f000087
:1017f800ae1f0000c31f0000d71f0000eb1f000032
:101808000020000014200000282000003d200000d7
:1018180051200000662000007a2000008e20000081
:10182800a3200000b7200000cc200000e02000002a
:10183800f4200000092100001d21000031210000d2
:10184800462100005a2100006f210000832100007a
:1018580098210000ac210000c0210000d521000023
:10186800e9210000fe2100001222000027220000ca
:101878003b22000050220000642200007922000070
:101888008d220000a2220000b6220000cb22000018
:10189800e0220000f4220000092300001d230000bc
:1018a80032230000472300005b2300007023000060
:1018b8008523000099230000ae230000c323000005
:1018c800d7230000ec2300000124000016240000a8
:1018d8002a2400003f24000054240000692400004a
:1018e8007e24000093240000a8240000bd240000ea
:1018f800d1240000e6240000fb240000102500008d
:10190800252500003b250000502500006525000026
:101918007a2500008f250000a4250000b9250000c5
:10192800cf250000e4250000f92500000e26000060
:1019380024260000392600004e26000064260000f8
:10194800792600008f260000a4260000ba26000091
:10195800cf260000e5260000fa2600001027000028
:10196800262700003b2700005127000067270000ba
:101978007d27000093270000a9270000be2700004c
:10198800d4270000ea2700000028000016280000dd
:101998002d28000043280000592800006f28000067
:1019a800852800009c280000b2280000c9280000f3
:1019b800df280000f52800000c290000232900007a
:1019c8003929000050290000672900007d290000fe
:1019d80094290000ab290000c2290000d929000081
:1019e800f0290000072a00001e2a0000352a0000fe
:1019f8004d2a0000642a00007b2a0000932a000078
:101a0800aa2a0000c22a0000da2a0000f12a0000ef
:101a1800092b0000212b0000392b0000512b00005e
:101a2800692b0000812b0000992b0000b12b0000ce
:101a3800c92b0000e22b0000fa2b0000132c000039
:101a48002b2c0000442c00005d2c0000762c00009c
:101a58008e2c0000a72c0000c12c0000da2c0000fe
:101a6800f32c00000c2d0000262d00003f2d000057
:101a7800592d0000732d00008d2d0000a72d0000aa
:101a8800c12d0000db2d0000f52d00000f2e0000f9
:101a98002a2e0000442e00005f2e00007a2e00003f
:101aa800952e0000b02e0000cb2e0000e62e000080
:101ab800022f00001d2f0000392f0000552f0000b5
:101ac800712f00008d2f0000a92f0000c62f0000e5
:101ad800e22f0000ff2f00001c300000393000000a
:101ae800563000007430000091300000af30000024
:101af800cd300000eb300000093100002831000033
:101b0800463100006531000084310000a431000036
:101b1800c3310000e331000003320000233200002b
:101b2800443200006532000086320000a73200000f
:101b3800c9320000ea3200000d3300002f330000e4
:101b4800523300007533000098330000bc330000a6
:101b5800e0330000053400002a3400004f34000050
:101b6800753400009b340000c2340000e9340000e2
:101b78001035000038350000613500008a35000056
:101b8800b4350000de3500000936000035360000a7
:101b9800623600008f360000bd360000ec360000cb
:101ba8001b3700004c3700007e370000b0370000bc
:101bb800e43700001a380000503800008838000068
:101bc800c2380000fd3800003b3900007a390000b7
:101bd800bc390000013a0000493a0000953a00007b
:101be800e43a0000393b0000943b0000f73b00005a
:101bf800643c0000e03c0000733d0000ff3f000033
:101c0800ff3f000000000000000100006a01000022
:101c1800bb010000000200003c020000730200004b
:101c2800a5020000d4020000000300002a030000ff
:101c380051030000770300009b030000be0300006f
:101c4800df03000000040000200400003e04000040
:101c58005c0400007904000095040000b104000051
:101c6800cc040000e604000000050000190500008f
:101c7800320500004b050000630500007a050000ee
:101c880091050000a8050000bf050000d50500006b
:101c9800eb05000000060000150600002a060000fb
:101ca8003f06000053060000670600007b060000a0
:101cb8008f060000a2060000b5060000c806000056
:101cc800db060000ee060000000700001207000017
:101cd80024070000360700004807000059070000e5
:101ce8006b0700007c0700008d0700009e070000be
:101cf800ae070000bf070000cf070000e0070000a4
:101d0800f00700000008000010080000200800008c
:101d18002f0800003f0800004e0800005e08000081
:101d28006d0800007c0800008b0800009a0800007d
:101d3800a9080000b8080000c6080000d50800007f
:101d4800e3080000f2080000000900000e09000086
:101d58001c0900002a090000380900004609000093
:101d680054090000610900006f0900007d090000a6
:101d78008a09000097090000a5090000b2090000bf
:101d8800bf090000cc090000d9090000e6090000dd
:101d9800f3090000000a00000d0a0000190a0000fb
:101da800260a0000330a00003f0a00004c0a00001f
:101db800580a0000640a0000710a00007d0a000049
:101dc800890a0000950a0000a10a0000ad0a000077
:101dd800b90a0000c50a0000d10a0000dd0a0000a7
:101de800e90a0000f40a0000000b00000c0b0000d8
:101df800170b0000230b00002e0b00003a0b00000d
:101e0800450b0000500b00005c0b0000670b000046
:101e1800720b00007d0b0000880b0000930b000084
:101e28009e0b0000a90b0000b40b0000bf0b0000c4
:101e3800ca0b0000d50b0000e00b0000eb0b000004
:101e4800f50b0000000c00000b0c0000150c000046
:101e5800200c00002a0c0000350c00003f0c00008c
:101e68004a0c0000540c00005f0c0000690c0000d4
:101e7800730c00007d0c0000880c0000920c000020
:101e88009c0c0000a60c0000b00c0000ba0c00006e
:101e9800c40c0000ce0c0000d80c0000e20c0000be
:101ea800ec0c0000f60c0000000d00000a0d00000c
:101eb800140d00001d0d0000270d0000310d00005d
:101ec8003b0d0000440d00004e0d0000570d0000b2
:101ed800610d00006b0d0000740d00007e0d000008
:101ee800870d0000910d00009a0d0000a30d000061
:101ef800ad0d0000b60d0000bf0d0000c90d0000bb
:101f0800d20d0000db0d0000e40d0000ee0d000016
:101f1800f70d0000000e0000090e0000120e000070
:101f28001b0e0000240e00002d0e0000360e0000cf
:101f38003f0e0000480e0000510e00005a0e00002f
:101f4800630e00006c0e0000750e00007e0e00008f
:101f5800870e00008f0e0000980e0000a10e0000f2
:101f6800aa0e0000b20e0000bb0e0000c40e000056
:101f7800cc0e0000d50e0000de0e0000e60e0000bc
:101f8800ef0e0000f70e0000000f0000080f000021
:101f9800110f0000190f0000220f00002a0f000087
:101fa800330f00003b0f0000440f00004c0f0000ef
:101fb800540f00005d0f0000650f00006d0f00005a
:101fc800760f00007e0f0000860f00008e0f0000c5
:101fd800970f00009f0f0000a70f0000af0f000031
:101fe800b70f0000bf0f0000c80f0000d00f00009f
:101ff800d80f0000e00f0000e80f0000f00f00000d
:10200800001000000000000000100000a1160000f1
:10201800b61b000000200000c72300003127000085
:10202800552a0000412d00000030000098320000c1
:10203800113500006d370000b0390000de3b0000ac
:10204800f73d000000400000f8410000e2430000b6
:10205800be4500008e470000524900000c4b0000ae
:10206800bb4c0000624e000000500000955100007b
:1020780023530000aa54000029560000a25700006c
:1020880015590000825a0000e95b00004b5d000012
:10209800a85e00000060000053610000a16200001b
:1020a800eb6300003165000073660000b167000053
:1020b800eb680000216a0000546b0000846c00008b
:1020c800b06d0000d96e00000070000023710000a0
:1020d80043720000607300007b7400009375000079
:1020e800a8760000bb770000cc780000da79000001
:1020f800e57a0000ef7b0000f67c0000fb7d000025
:10210800fe7e000000800000ff800000fc810000cf
:10211800f7820000f0830000e7840000dd850000fe
:10212800d1860000c3870000b4880000a38900009e
:10213800908a00007c8b0000668c00004e8d0000a9
:10214800358e00001b8f0000ff8f0000e29000001a
:10215800c4910000a49200008393000060940000e2
:102168003c95000017960000f1960000c997000002
:10217800a1980000779900004c9a0000209b00006d
:10218800f29b0000c49c0000949d0000649e000027
:10219800329f0000ff9f0000cca0000097a1000024
:1021a80061a200002ba30000f3a30000baa4000062
:1021b80081a5000046a600000ba70000cfa70000dd
:1021c80091a8000053a9000014aa0000d5aa000095
:1021d80094ab000053ac000010ad0000cdad000082
:1021e80089ae000045af0000ffaf0000b9b00000a5
:1021f80072b100002ab20000e2b2000099b30000f8
:102208004fb4000004b50000b9b500006db6000079
:1022180020b70000d3b7000085b8000036b9000029
:10222800e6b9000096ba000046bb0000f4bb000007
:10223800a2bc000050bd0000fdbd0000a9be00000a
:1022480054bf0000ffbf0000aac0000053c1000037
:10225800fdc10000a5c200004dc30000f5c3000089
:102268009cc4000042c50000e8c500008dc60000ff
:1022780032c70000d6c700007ac800001dc9000098
:10228800c0c9000062ca000004cb0000a5cb000052
:1022980045cc0000e6cc000085cd000024ce00002f
:1022a800c3ce000061cf0000ffcf00009cd000002b
:1022b80039d10000d6d1000072d200000dd3000041
:1022c800a8d3000043d40000ddd4000077d5000077
:1022d80010d60000a9d6000041d70000d9d70000c9
:1022e80071d8000008d900009fd9000035da000035
:1022f800cbda000061db0000f6db00008bdc0000bd
:102308001fdd0000b3dd000047de0000dade00005c
:102318006ddf0000ffdf000091e0000023e1000016
:10232800b4e1000045e20000d6e2000066e30000e8
:10233800f6e3000086e4000015e50000a4e50000cf
:1023480032e60000c0e600004ee70000dce70000cf
:1023580069e80000f6e8000082e900000eea0000e3
:102368009aea000026eb0000b1eb00003cec00000c
:10237800c6ec000051ed0000daed000064ee00004c
:10238800edee000076ef0000ffef000087f00000a0
:1023980010f1000097f100001ff20000a6f2000003
:1023a8002df30000b3f300003af40000c0f400007d
:1023b80046f50000cbf5000050f60000d5f6000009
:1023c8005af70000def7000062f80000e6f80000a7
:1023d80069f90000edf9000070fa0000f2fa000057
:1023e80075fb0000f7fb000079fc0000fafc000018
:1023f8007cfd0000fdfd00007efe0000fffe0000e9
:10240800ffff0000ffff000000c000008cc20000ba
:102418009bc300006ac4000019c50000b3c50000d2
:102428003fc60000bfc6000037c70000a7c70000ae
:1024380011c8000076c80000d7c8000034c90000e1
:102448008dc90000e3c9000037ca000088ca00002f
:10245800d6ca000023cb00006dcb0000b6cb00002d
:10246800fdcb000043cc000087cc0000c9cc0000a5
:102478000bcd00004bcd00008acd0000c8cd000078
:1024880005ce000041ce00007cce0000b6ce000094
:10249800efce000027cf00005fcf000096cf0000ee
:1024a800cccf000002d0000037d000006bd0000075
:1024b8009fd00000d2d0000004d1000036d1000027
:1024c80068d1000098d10000c9d10000f9d10000fe
:1024d80028d2000057d2000086d20000b4d20000f3
:1024e800e2d200000fd300003cd3000069d3000003
:1024f80095d30000c1d30000edd3000018d400002c
:1025080043d400006dd4000097d40000c1d400006b
:10251800ebd4000014d500003dd5000066d50000be
:102528008fd50000b7d50000dfd5000007d6000022
:102538002ed6000055d600007cd60000a3d6000099
:10254800c9d60000f0d6000016d700003cd700001e
:1025580061d7000087d70000acd70000d1d70000b2
:10256800f6d700001ad800003fd8000063d8000052
:1025780087d80000abd80000cfd80000f2d8000000
:1025880016d9000039d900005cd900007fd90000b5
:10259800a1d90000c4d90000e6d9000009da00007a
:1025a8002bda00004dda00006eda000090da000045
:1025b800b2da0000d3da0000f4da000015db00001c
:1025c80036db000057db000078db000098db0000fa
:1025d800b9db0000d9db0000f9db000019dc0000e2
:1025e80039dc000059dc000079dc000098dc0000d0
:1025f800b8dc0000d7dc0000f7dc000016dd0000c6
:1026080035dd000054dd000073dd000091dd0000c1
:10261800b0dd0000cfdd0000eddd00000bde0000c6
:102628002ade000048de000066de000084de0000ce
:10263800a2de0000bfde0000ddde0000fbde0000e1
:1026480018df000036df000053df000070df0000f5
:102658008ddf0000abdf0000c8df0000e5df000011
:1026680001e000001ee000003be0000057e0000031
:1026780074e0000090e00000ade00000c9e0000058
:10268800e5e0000002e100001ee100003ae1000080
:1026980056e1000071e100008de10000a9e10000b1
:1026a800c5e10000e0e10000fce1000017e20000e5
:1026b80033e200004ee2000069e2000084e200001c
:1026c800a0e20000bbe20000d6e20000f1e2000058
:1026d8000ce3000026e3000041e300005ce3000097
:1026e80077e3000091e30000ace30000c6e30000dc
:1026f800e1e30000fbe3000016e4000030e4000022
:102708004ae4000064e400007ee4000098e400006d
:10271800b2e40000cce40000e6e4000000e50000bc
:102728001ae5000034e500004de5000067e500000b
:1027380081e500009ae50000b4e50000cde5000061
:10274800e7e5000000e6000019e6000033e60000b7
:102758004ce6000065e600007ee6000098e6000012
:10276800b1e60000cae60000e3e60000fce600006f
:1027780014e700002de7000046e700005fe70000cf
:1027880078e7000090e70000a9e70000c2e7000032
:10279800dae70000f3e700000be8000024e8000097
:1027a8003ce8000055e800006de8000085e80000fe
:1027b8009de80000b6e80000cee80000e6e800006a
:1027c800fee8000016e900002ee9000046e90000d6
:1027d8005ee9000076e900008ee90000a6e9000045
:1027e800bee90000d6e90000eee9000005ea0000b5
:1027f8001dea000035ea00004cea000064ea000027
:102808007cea000093ea0000abea0000c2ea00009c
:10281800daea0000f1ea000009eb000020eb000012
:1028280037eb00004feb000066eb00007deb00008b
:1028380095eb0000aceb0000c3eb0000daeb000006
:10284800f1eb000008ec00001fec000036ec000083
:102858004eec000064ec00007bec000092ec000001
:10286800a9ec0000c0ec0000d7ec0000eeec000082
:1028780005ed00001ced000032ed000049ed000000
:1028880060ed000076ed00008ded0000a4ed000085
:10289800baed0000d1ed0000e8ed0000feed00000b
:1028a80015ee00002bee000042ee000058ee00008e
:1028b8006eee000085ee00009bee0000b2ee000018
:1028c800c8ee0000deee0000f5ee00000bef0000a1
:1028d80021ef000037ef00004eef000064ef00002a
:1028e8007aef000090ef0000a6ef0000bcef0000b8
:1028f800d3ef0000e9ef0000ffef000015f0000043
:102908002bf0000041f0000057f000006df00000cf
:1029180083f0000099f00000aef00000c4f0000061
:10292800daf00000f0f0000006f100001cf10000f1
:1029380032f1000047f100005df1000073f1000082
:1029480089f100009ef10000b4f10000caf1000016
:10295800dff10000f5f100000bf2000020f20000aa
:1029680036f200004bf2000061f2000077f200003e
:102978008cf20000a2f20000b7f20000cdf20000d5
:10298800e2f20000f8f200000df3000023f300006b
:1029980038f300004df3000063f3000078f3000003
:1029a8008df30000a3f30000b8f30000cef300009d
:1029b800e3f30000f8f300000df4000023f4000036
:1029c80038f400004df4000062f4000078f40000d0
:1029d8008df40000a2f40000b7f40000ccf400006d
:1029e800e2f40000f7f400000cf5000021f5000007
:1029f80036f500004bf5000060f5000075f50000a5
:102a08008af500009ff50000b5f50000caf5000042
:102a1800dff50000f4f5000009f600001ef60000de
:102a280033f6000048f600005df6000071f600007d
:102a380086f600009bf60000b0f60000c5f6000020
:102a4800daf60000eff6000004f7000019f70000be
:102a58002ef7000042f7000057f700006cf700005f
:102a680081f7000096f70000abf70000bff7000001
:102a7800d4f70000e9f70000fef7000012f80000a4
:102a880027f800003cf8000051f8000065f8000045
:102a98007af800008ff80000a4f80000b8f80000e9
:102aa800cdf80000e2f80000f6f800000bf900008d
:102ab80020f9000034f9000049f900005ef900002f
:102ac80072f9000087f900009cf90000b0f90000d5
:102ad800c5f90000d9f90000eef9000003fa00007a
:102ae80017fa00002cfa000040fa000055fa00001e
:102af8006afa00007efa000093fa0000a7fa0000c4
:102b0800bcfa0000d0fa0000e5fa0000f9fa00006b
:102b18000efb000022fb000037fb00004bfb00000f
:102b280060fb000074fb000089fb00009dfb0000b7
:102b3800b2fb0000c6fb0000dbfb0000effb00005f
:102b480004fc000018fc00002dfc000041fc000003
:102b580056fc00006afc00007ffc000093fc0000ab
:102b6800a7fc0000bcfc0000d0fc0000e5fc000055
:102b7800f9fc00000efd000022fd000036fd0000fb
:102b88004bfd00005ffd000074fd000088fd0000a3
:102b98009dfd0000b1fd0000c5fd0000dafd00004c
:102ba800eefd000003fe000017fe00002bfe0000f3
:102bb80040fe000054fe000068fe00007dfe00009c
:102bc80091fe0000a6fe0000bafe0000cefe000046
:102bd800e3fe0000f7fe00000cff000020ff0000ed
:102be80034ff000049ff00005dff000071ff000096
:102bf80086ff00009aff0000afff0000c3ff00003f
:102c0800d7ff0000ecff00000000000014000000e7
:102c1800290000003d00000051000000660000008f
:102c28007a0000008f000000a3000000b700000039
:102c3800cc000000e0000000f400000009010000e2
:102c48001d01000032010000460100005a01000089
:102c58006f0100008301000098010000ac01000032
:102c6800c0010000d5010000e9010000fd010000dd
:102c780012020000260200003b0200004f02000082
:102c880063020000780200008c020000a10200002c
:102c9800b5020000ca020000de020000f2020000d5
:102ca800070300001b03000030030000440300007a
:102cb800590300006d030000810300009603000023
:102cc800aa030000bf030000d3030000e8030000cc
:102cd800fc03000011040000250400003a04000071
:102ce8004e04000063040000770400008c04000018
:102cf800a0040000b5040000c9040000de040000c0
:102d0800f2040000070500001b0500003005000064
:102d180044050000590500006d050000820500000b
:102d280096050000ab050000c0050000d4050000b2
:102d3800e9050000fd050000120600002706000056
:102d48003b060000500600006406000079060000fb
:102d58008e060000a2060000b7060000cc060000a0
:102d6800e0060000f50600000a0700001e07000044
:102d780033070000480700005c07000071070000e7
:102d8800860700009b070000af070000c40700008b
:102d9800d9070000ee07000002080000170800002d
:102da8002c08000041080000550800006a080000cf
:102db8007f08000094080000a9080000be08000071
:102dc800d2080000e7080000fc0800001109000014
:102dd800260900003b0900005009000065090000b1
:102de8007a0900008f090000a3090000b809000053
:102df800cd090000e2090000f70900000c0a0000f4
:102e0800210a0000360a00004b0a0000610a00008f
:102e1800760a00008b0a0000a00a0000b50a00002c
:102e2800ca0a0000df0a0000f40a0000090b0000cb
:102e38001e0b0000340b0000490b00005e0b000065
:102e4800730b0000880b00009e0b0000b30b000002
:102e5800c80b0000dd0b0000f30b0000080c00009d
:102e68001d0c0000320c0000480c00005d0c000036
:102e7800730c0000880c00009d0c0000b30c0000cf
:102e8800c80c0000dd0c0000f30c0000080d000069
:102e98001e0d0000330d0000490d00005e0d0000fe
:102ea800740d0000890d00009f0d0000b50d000095
:102eb800ca0d0000e00d0000f50d00000b0e00002b
:102ec800210e0000360e00004c0e0000620e0000bd
:102ed800770e00008d0e0000a30e0000b90e000052
:102ee800ce0e0000e40e0000fa0e0000100f0000e5
:102ef800260f00003c0f0000520f0000670f000073
:102f08007d0f0000930f0000a90f0000bf0f000005
:102f1800d50f0000eb0f0000011000001710000093
:102f28002d100000441000005a100000701000001e
:102f3800861000009c100000b2100000c9100000ac
:102f4800df100000f51000000b1100002211000036
:102f5800381100004e110000651100007b110000bf
:102f680092110000a8110000be110000d511000048
:102f7800eb11000002120000181200002f120000ce
:102f8800461200005c120000731200008a12000052
:102f9800a0120000b7120000ce120000e4120000d8
:102fa800fb12000012130000291300004013000058
:102fb800571300006e130000851300009c130000d7
:102fc800b2130000ca130000e1130000f813000058
:102fd8000f140000261400003d14000054140000d3
:102fe8006b140000831400009a140000b114000050
:102ff800c9140000e0140000f71400000f150000c9
:10300800261500003e150000551500006d1500003e
:10301800841500009c150000b4150000cb150000b5
:10302800e3150000fb150000121600002a16000028
:10303800421600005a160000721600008a16000098
:10304800a2160000ba160000d2160000ea16000008
:10305800021700001a170000321700004a17000074
:10306800631700007b17000093170000ab170000e0
:10307800c4170000dc170000f51700000d18000049
:10308800261800003e1800005718000070180000ad
:1030980088180000a1180000ba180000d318000012
:1030a800ec180000041900001d1900003619000072
:1030b8004f19000068190000821900009b190000d0
:1030c800b4190000cd190000e7190000001a00002b
:1030d800191a0000331a00004c1a0000661a000082
:1030e8007f1a0000991a0000b31a0000cc1a0000d9
:1030f800e61a0000001b00001a1b0000341b000029
:103108004e1b0000681b0000821b00009c1b000077
:10311800b61b0000d01b0000ea1b0000051c0000c5
:103128001f1c00003a1c0000541c00006f1c00000b
:10313800891c0000a41c0000bf1c0000da1c000051
:10314800f41c00000f1d00002a1d0000451d000092
:10315800601d00007c1d0000971d0000b21d0000ce
:10316800cd1d0000e91d0000041e0000201e000007
:103178003b1e0000571e0000731e00008f1e00003b
:10318800aa1e0000c61e0000e21e0000fe1e00006f
:103198001b1f0000371f0000531f0000701f000096
:1031a8008c1f0000a91f0000c51f0000e21f0000bf
:1031b800ff1f00001b2000003820000055200000e1
:1031c8007320000090200000ad200000ca200000fd
:1031d800e820000005210000232100004121000013
:1031e8005e2100007c2100009a210000b821000027
:1031f800d6210000f5210000132200003122000032
:10320800502200006f2200008d220000ac22000036
:10321800cb220000ea220000092300002923000035
:10322800482300006823000087230000a72300002c
:10323800c7230000e723000007240000272400001c
:10324800472400006824000088240000a924000006
:10325800ca240000eb2400000c2500002d250000e6
:103268004e2500007025000092250000b3250000bf
:10327800d5250000f72500001a2600003c2600008e
:103288005f26000081260000a4260000c726000053
:10329800ea2600000e27000031270000552700000d
:1032a800792700009d270000c1270000e6270000bd
:1032b8000a2800002f280000542800007928000060
:1032c8009f280000c4280000ea28000010290000f8
:1032d800372900005d29000084290000ab2900007f
:1032e800d2290000f9290000212a0000492a0000fb
:1032f800712a00009a2a0000c32a0000ec2a000064
:10330800152b00003f2b0000692b0000932b0000b9
:10331800bd2b0000e82b0000132c00003f2c000000
:103328006b2c0000972c0000c42c0000f12c00002e
:103338001e2d00004c2d00007a2d0000a92d000044
:10334800d82d0000072e0000372e0000682e000040
:10335800982e0000ca2e0000fc2e00002e2f000020
:10336800612f0000952f0000c92f0000fe2f0000dc
:10337800343000006a300000a1300000d93000006d
:10338800113100004a31000084310000bf310000d3
:10339800fb3100003832000076320000b532000000
:1033a800f53200003733000079330000bd330000e8
:1033b800033400004a34000093340000dd34000078
:1033c8002a35000078350000c93500001d36000098
:1033d80073360000cc360000293700008a37000019
:1033e800ef37000059380000c938000041390000a3
:1033f800c13900004d3a0000e73a0000963b000052
:10340800653c0000743d0000743d000000e00000d1
:1034180015e0000029e000003ee0000052e0000056
:1034280067e000007ce0000091e00000a6e00000fa
:10343800bbe00000d0e00000e5e00000fbe0000099
:1034480010e1000025e100003be1000051e100002f
:1034580066e100007ce1000092e10000a8e10000c4
:10346800bee10000d4e10000eae1000001e2000052
:1034780017e200002ee2000044e200005be20000d8
:1034880072e2000089e20000a0e20000b7e200005a
:10349800cee20000e5e20000fce2000014e30000d8
:1034a8002be3000043e300005ae3000072e300004e
:1034b8008ae30000a2e30000bae30000d2e30000c0
:1034c800eae3000003e400001be4000033e400002a
:1034d8004ce4000065e400007de4000096e4000090
:1034e800afe40000c8e40000e2e40000fbe40000f0
:1034f80014e500002ee5000047e5000061e5000046
:103508007ae5000094e50000aee50000c8e500009b
:10351800e2e50000fde5000017e6000031e60000e6
:103528004ce6000066e6000081e600009ce600002c
:10353800b7e60000d2e60000ede6000008e700006c
:1035480024e700003fe700005ae7000076e70000a4
:1035580092e70000aee70000cae70000e6e70000d7
:1035680002e800001ee800003ae8000057e8000002
:1035780073e8000090e80000ade80000c9e800002a
:10358800e6e8000003e9000021e900003ee9000048
:103598005be9000079e9000096e90000b4e9000061
:1035a800d2e90000efe900000dea00002bea000074
:1035b8004aea000068ea000086ea0000a5ea00007e
:1035c800c3ea0000e2ea000001eb000020eb000083
:1035d8003feb00005eeb00007deb00009ceb000081
:1035e800bceb0000dbeb0000fbeb00001bec000079
:1035f8003aec00005aec00007aec00009bec00006a
:10360800bbec0000dbec0000fcec00001ced000053
:103618003ded00005eed00007eed00009fed000036
:10362800c0ed0000e2ed000003ee000024ee000013
:1036380046ee000067ee000089ee0000abee0000e9
:10364800ccee0000eeee000010ef000033ef0000bb
:1036580055ef000077ef00009aef0000bcef000084
:10366800dfef000001f0000024f0000047f0000048
:103678006af000008df00000b1f00000d4f0000006
:10368800f7f000001bf100003ef1000062f10000bd
:1036980086f10000aaf10000cef10000f2f100006e
:1036a80016f200003af200005ef2000083f2000019
:1036b800a7f20000ccf20000f0f2000015f30000c1
:1036c8003af300005ff3000084f30000a9f3000060
:1036d800cef30000f3f3000019f400003ef40000fc
:1036e80063f4000089f40000aff40000d4f4000093
:1036f800faf4000020f5000046f500006cf5000023
:1037080092f50000b8f50000dff5000005f60000ae
:103718002bf6000052f6000078f600009ff6000035
:10372800c5f60000ecf6000013f700003af70000b9
:1037380061f7000088f70000aff70000d6f7000037
:10374800fdf7000024f800004bf8000073f80000b3
:103758009af80000c2f80000e9f8000011f900002a
:1037680038f9000060f9000088f90000aff900009e
:10377800d7f90000fff9000027fa00004ffa00000f
:1037880077fa00009ffa0000c7fa0000effa00007d
:1037980017fb00003ffb000067fb000090fb0000e8
:1037a800b8fb0000e0fb000009fc000031fc000051
:1037b80059fc000082fc0000aafc0000d3fc0000b9
:1037c800fbfc000024fd00004cfd000075fd00001e
:1037d8009efd0000c6fd0000effd000017fe000082
:1037e80040fe000069fe000091fe0000bafe0000e5
:1037f800e3fe00000cff000034ff00005dff000046
:1038080086ff0000afff0000d7ff000000000000a7
:1038180029000000510000007a000000a300000009
:10382800cc000000f40000001d010000460100006b
:103838006f01000097010000c0010000e9010000cd
:10384800110200003a020000620200008b02000030
:10385800b4020000dc020000050300002d03000094
:10386800560300007e030000a7030000cf030000fa
:10387800f703000020040000480400007004000062
:1038880099040000c1040000e904000011050000cb
:10389800390500006105000089050000b105000038
:1038a800d9050000010600002906000051060000a5
:1038b80078060000a0060000c8060000ef06000019
:1038c800170700003e070000660700008d0700008c
:1038d800b5070000dc070000030800002a08000004
:1038e80051080000780800009f080000c608000082
:1038f800ed080000140900003b0900006109000000
:1039080088090000ae090000d5090000fb09000085
:10391800210a0000480a00006e0a0000940a00000c
:10392800ba0a0000e00a0000060b00002c0b000099
:10393800510b0000770b00009d0b0000c20b00002c
:10394800e70b00000d0c0000320c0000570c0000c3
:103958007c0c0000a10c0000c60c0000eb0c000061
:10396800100d0000340d0000590d00007d0d000001
:10397800a20d0000c60d0000ea0d00000e0e0000aa
:10398800320e0000560e00007a0e00009e0e000057
:10399800c20e0000e50e0000090f00002c0f000009
:1039a8004f0f0000730f0000960f0000b90f0000c2
:1039b800dc0f0000ff0f0000211000004410000081
:1039c8006610000089100000ab100000cd10000048
:1039d800f010000012110000341100005511000011
:1039e8007711000099110000ba110000dc110000e5
:1039f800fd1100001e1200004012000061120000bc
:103a080082120000a2120000c3120000e41200009b
:103a1800041300002513000045130000651300007f
:103a280086130000a6130000c6130000e51300006b
:103a3800051400002514000044140000641400005c
:103a480083140000a2140000c1140000e014000058
:103a5800ff1400001e1500003d1500005b15000056
:103a68007a15000098150000b6150000d51500005d
:103a7800f3150000111600002e1600004c16000069
:103a88006a16000087160000a5160000c21600007e
:103a9800df160000fd1600001a1700003717000097
:103aa80053170000701700008d170000a9170000b9
:103ab800c6170000e2170000fe1700001a180000e1
:103ac80036180000521800006e1800008a1800000e
:103ad800a6180000c1180000dc180000f818000043
:103ae800131900002e19000049190000641900007c
:103af8007f1900009a190000b4190000cf190000be
:103b0800e9190000031a00001e1a0000381a000004
:103b1800521a00006c1a0000861a00009f1a000052
:103b2800b91a0000d21a0000ec1a0000051b0000a8
:103b38001e1b0000381b0000511b00006a1b000000
:103b4800831b00009b1b0000b41b0000cd1b000062
:103b5800e51b0000fd1b0000161c00002e1c0000c9
:103b6800461c00005e1c0000761c00008e1c000035
:103b7800a61c0000bd1c0000d51c0000ec1c0000a9
:103b8800041d00001b1d0000321d0000491d00001f
:103b9800601d0000771d00008e1d0000a51d00009f
:103ba800bc1d0000d21d0000e91d0000ff1d000023
:103bb800161e00002c1e0000421e0000581e0000a9
:103bc8006e1e0000841e00009a1e0000af1e00003a
:103bd800c51e0000db1e0000f01e0000051f0000cf
:103be8001b1f0000301f0000451f00005a1f000067
:103bf8006f1f0000841f0000991f0000ae1f000007
:103c0800c21f0000d71f0000eb1f0000eb1f0000c1
:103c180001800000038000000b8000001780000076
:103c2800288000003f8000005a8000007a80000051
:103c38009f800000c9800000f78000002b810000f1
:103c480064810000a1810000e38100002b82000054
:103c580077820000c78200001d830000788300007f
:103c6800d78300003b840000a48400001285000074
:103c780084850000fb85000077860000f786000039
:103c88007c870000068800009588000028890000cd
:103c9800bf8900005b8a0000fc8a0000a18b00003d
:103ca8004b8c0000f98c0000ac8d0000638e000086
:103cb8001e8f0000de8f0000a29000006a910000b5
:103cc8003792000008930000dd930000b6940000ce
:103cd80093950000759600005a97000044980000dc
:103ce80031990000239a0000189b0000129c0000e4
:103cf8000f9d0000109e0000159f00001da00000f1
:103d080029a1000039a200004da3000064a400000e
:103d18007ea500009ca60000bea70000e3a8000046
:103d28000baa000037ab000065ac000098ad00009e
:103d3800cdae000005b0000041b100007fb2000028
:103d4800c1b3000005b500004cb6000097b70000ed
:103d5800e4b8000033ba000086bb0000dbbc0000fa
:103d680032be00008dbf0000e9c0000048c200005c
:103d7800aac300000ec5000074c60000dcc700001e
:103d880046c90000b3ca000021cc000092cd000053
:103d980005cf000079d00000efd1000067d3000004
:103da800e1d400005dd60000dad7000058d9000041
:103db800d8da00005adc0000dddd000061df000019
:103dc800e6e000006de20000f5e300007ee500009b
:103dd80007e7000092e800001eea0000abeb0000d5
:103de80038ed0000c6ee000055f00000e4f10000d8
:103df80074f3000005f5000096f6000027f80000af
:103e0800b8f900004afb0000dcfc00006efe000070
:103e1800000000009201000024030000b604000026
:103e280048060000d90700006a090000fb0a0000e4
:103e38008c0c00001c0e0000ab0f00003a110000b3
:103e4800c812000055140000e21500006e170000ab
:103e5800f9180000821a00000b1c0000931d0000d6
:103e68001a1f00009f20000023220000a623000044
:103e780028250000a826000026280000a329000005
:103e88001f2b0000992c0000112e0000872f000026
:103e9800fb3000006e320000df3300004d350000bb
:103ea800ba360000243800008c390000f23a0000cd
:103eb800563c0000b83d0000173f0000734000006a
:103ec800ce410000254300007a440000cd450000a3
:103ed8001c47000069480000b4490000fb4a000084
:103ee8003f4c0000814d0000bf4e0000fb4f00001a
:103ef80033510000685200009b530000c954000071
:103f0800f55500001d570000425800006459000094
:103f1800825a00009c5b0000b35c0000c75d000093
:103f2800d75e0000e35f0000eb600000f061000076
:103f3800f1620000ee630000e8640000dd65000047
:103f4800cf660000bc670000a66800008b6900000f
:103f58006d6a00004a6b0000236c0000f86c0000da
:103f6800c96d0000966e00005e6f000022700000b0
:103f7800e27000009d710000547200000773000099
:103f8800b57300005f74000004750000a57500009b
:103f980041760000d87600006b770000fa770000c1
:103fa800847800000979000089790000057a00000a
:103fb8007c7a0000ee7a00005c7b0000c57b000084
:103fc800297c0000887c0000e37c0000397d00002b
:103fd800897d0000d57d00001d7e00005f7e000009
:103fe8009c7e0000d57e0000097f0000377f00001e
:103ff800617f0000867f0000a67f0000c17f00006f
:10400800d87f0000e97f0000f57f0000fd7f0000f9
:10401800ff7f0000fd7f0000f57f0000e97f0000c2
:10402800d87f0000c17f0000a67f0000867f0000c7
:10403800617f0000377f0000097f0000d57e000007
:104048009c7e00005f7e00001d7e0000d57d000084
:10405800897d0000397d0000e37c0000887c000039
:10406800297c0000c57b00005c7b0000ee7a000024
:104078007c7a0000057a000089790000097900003f
:1040880084780000fa7700006b770000d87600008b
:1040980041760000a5750000047500005f740000fb
:1040a800b573000007730000547200009d71000092
:1040b800e2700000227000005e6f0000966e000043
:1040c800c96d0000f86c0000236c00004a6b00000a
:1040d8006d6a00008b690000a6680000bc670000dc
:1040e800cf660000dd650000e8640000ee630000b4
:1040f800f1620000f0610000eb600000e35f000087
:10410800d75e0000c75d0000b35c00009c5b000048
:10411800825a000064590000425800001d570000f0
:10412800f5550000c95400009b5300006852000078
:1041380033510000fb4f0000bf4e0000814d0000ce
:104148003f4c0000fb4a0000b449000069480000e9
:104158001c470000cd4500007a44000025430000bc
:10416800ce41000073400000173f0000b83d00003a
:10417800563c0000f23a00008c3900002438000058
:10418800ba3600004d350000df3300006e32000003
:10419800fb300000872f0000112e0000992c000032
:1041a8001f2b0000a329000026280000a8260000d5
:1041b80028250000a6230000232200009f200000dd
:1041c8001a1f0000931d00000b1c0000821a00003b
:1041d800f91800006e170000e215000055140000e1
:1041e800c81200003a110000ab0f00001c0e0000be
:1041f8008c0c0000fb0a00006a090000d9070000c7
:1042080048060000b60400002403000092010000e4
:10421800000000006efe0000dcfc00004afb00000d
:10422800b8f9000027f8000096f6000005f5000030
:1042380074f30000e4f1000055f00000c6ee000041
:1042480038ed0000abeb00001eea000092e8000029
:1042580007e700007ee50000f5e300006de20000de
:10426800e6e0000061df0000dddd00005adc000050
:10427800d8da000058d90000dad700005dd600006f
:10428800e1d4000067d30000efd1000079d000002e
:1042980005cf000092cd000021cc0000b3ca000079
:1042a80046c90000dcc7000074c600000ec5000047
:1042b800aac3000048c20000e9c000008dbf00008a
:1042c80032be0000dbbc000086bb000033ba000031
:1042d800e4b8000097b700004cb6000005b5000030
:1042e800c1b300007fb2000041b1000005b000007a
:1042f800cdae000098ad000065ac000037ab000003
:104308000baa0000e3a80000bea700009ca60000be
:104318007ea5000064a400004da3000039a200009f
:1043280029a100001da00000159f0000109e00009c
:104338000f9d0000129c0000189b0000239a0000ab
:1043480031990000449800005a97000075960000c3
:1043580093950000b6940000dd93000008930000d8
:10436800379200006a910000a2900000de8f0000e2
:104378001e8f0000638e0000ac8d0000f98c0000d9
:104388004b8c0000a18b0000fc8a00005b8a0000b7
:10439800bf89000028890000958800000688000071
:1043a8007c870000f786000077860000fb85000008
:1043b8008485000012850000a48400003b8400006e
:1043c800d7830000788300001d830000c7820000a7
:1043d800778200002b820000e3810000a1810000a9
:1043e800648100002b810000f7800000c980000074
:1043f8009f8000007a8000005a8000003f80000003
:1044080028800000178000000b8000000380000057
:10441800000000006efe0000dcfc00004afb00000b
:10442800b8f9000027f8000096f6000005f500002e
:1044380074f30000e4f1000055f00000c6ee00003f
:1044480038ed0000abeb00001eea000092e8000027
:1044580007e700007ee50000f5e300006de20000dc
:10446800e6e0000061df0000dddd00005adc00004e
:10447800d8da000058d90000dad700005dd600006d
:10448800e1d4000067d30000efd1000079d000002c
:1044980005cf000092cd000021cc0000b3ca000077
:1044a80046c90000dcc7000074c600000ec5000045
:1044b800aac3000048c20000e9c000008dbf000088
:1044c80032be0000dbbc000086bb000033ba00002f
:1044d800e4b8000097b700004cb6000005b500002e
:1044e800c1b300007fb2000041b1000005b0000078
:1044f800cdae000098ad000065ac000037ab000001
:104508000baa0000e3a80000bea700009ca60000bc
:104518007ea5000064a400004da3000039a200009d
:1045280029a100001da00000159f0000109e00009a
:104538000f9d0000129c0000189b0000239a0000a9
:1045480031990000449800005a97000075960000c1
:1045580093950000b6940000dd93000008930000d6
:10456800379200006a910000a2900000de8f0000e0
:104578001e8f0000638e0000ac8d0000f98c0000d7
:104588004b8c0000a18b0000fc8a00005b8a0000b5
:10459800bf8900002889000095880000068800006f
:1045a8007c870000f786000077860000fb85000006
:1045b8008485000012850000a48400003b8400006c
:1045c800d7830000788300001d830000c7820000a5
:1045d800778200002b820000e3810000a1810000a7
:1045e800648100002b810000f7800000c980000072
:1045f8009f8000007a8000005a8000003f80000001
:1046080028800000178000000b8000000380000055
:1046180001800000038000000b800000178000006c
:10462800288000003f8000005a8000007a80000047
:104638009f800000c9800000f78000002b810000e7
:1046480064810000a1810000e38100002b8200004a
:1046580077820000c78200001d8300007883000075
:10466800d78300003b840000a4840000128500006a
:1046780084850000fb85000077860000f78600002f
:104688007c870000068800009588000028890000c3
:10469800bf8900005b8a0000fc8a0000a18b000033
:1046a8004b8c0000f98c0000ac8d0000638e00007c
:1046b8001e8f0000de8f0000a29000006a910000ab
:1046c8003792000008930000dd930000b6940000c4
:1046d80093950000759600005a97000044980000d2
:1046e80031990000239a0000189b0000129c0000da
:1046f8000f9d0000109e0000159f00001da00000e7
:1047080029a1000039a200004da3000064a4000004
:104718007ea500009ca60000bea70000e3a800003c
:104728000baa000037ab000065ac000098ad000094
:10473800cdae000005b0000041b100007fb200001e
:10474800c1b3000005b500004cb6000097b70000e3
:10475800e4b8000033ba000086bb0000dbbc0000f0
:1047680032be00008dbf0000e9c0000048c2000052
:10477800aac300000ec5000074c60000dcc7000014
:1047880046c90000b3ca000021cc000092cd000049
:1047980005cf000079d00000efd1000067d30000fa
:1047a800e1d400005dd60000dad7000058d9000037
:1047b800d8da00005adc0000dddd000061df00000f
:1047c800e6e000006de20000f5e300007ee5000091
:1047d80007e7000092e800001eea0000abeb0000cb
:1047e80038ed0000c6ee000055f00000e4f10000ce
:1047f80074f3000005f5000096f6000027f80000a5
:10480800b8f900004afb0000dcfc00006efe000066
:10481800000000009201000024030000b60400001c
:1048280048060000d90700006a090000fb0a0000da
:104838008c0c00001c0e0000ab0f00003a110000a9
:10484800c812000055140000e21500006e170000a1
:10485800f9180000821a00000b1c0000931d0000cc
:104868001a1f00009f20000023220000a62300003a
:1048780028250000a826000026280000a3290000fb
:104888001f2b0000992c0000112e0000872f00001c
:10489800fb3000006e320000df3300004d350000b1
:1048a800ba360000243800008c390000f23a0000c3
:1048b800563c0000b83d0000173f00007340000060
:1048c800ce410000254300007a440000cd45000099
:1048d8001c47000069480000b4490000fb4a00007a
:1048e8003f4c0000814d0000bf4e0000fb4f000010
:1048f80033510000685200009b530000c954000067
:10490800f55500001d57000042580000645900008a
:10491800825a00009c5b0000b35c0000c75d000089
:10492800d75e0000e35f0000eb600000f06100006c
:10493800f1620000ee630000e8640000dd6500003d
:10494800cf660000bc670000a66800008b69000005
:104958006d6a00004a6b0000236c0000f86c0000d0
:10496800c96d0000966e00005e6f000022700000a6
:10497800e27000009d71000054720000077300008f
:10498800b57300005f74000004750000a575000091
:1049980041760000d87600006b770000fa770000b7
:1049a800847800000979000089790000057a000000
:1049b8007c7a0000ee7a00005c7b0000c57b00007a
:1049c800297c0000887c0000e37c0000397d000021
:1049d800897d0000d57d00001d7e00005f7e0000ff
:1049e8009c7e0000d57e0000097f0000377f000014
:1049f800617f0000867f0000a67f0000c17f000065
:104a0800d87f0000e97f0000f57f0000fd7f0000ef
:104a1800ff7f0000fd7f0000f57f0000e97f0000b8
:104a2800d87f0000c17f0000a67f0000867f0000bd
:104a3800617f0000377f0000097f0000d57e0000fd
:104a48009c7e00005f7e00001d7e0000d57d00007a
:104a5800897d0000397d0000e37c0000887c00002f
:104a6800297c0000c57b00005c7b0000ee7a00001a
:104a78007c7a0000057a0000897900000979000035
:104a880084780000fa7700006b770000d876000081
:104a980041760000a5750000047500005f740000f1
:104aa800b573000007730000547200009d71000088
:104ab800e2700000227000005e6f0000966e000039
:104ac800c96d0000f86c0000236c00004a6b000000
:104ad8006d6a00008b690000a6680000bc670000d2
:104ae800cf660000dd650000e8640000ee630000aa
:104af800f1620000f0610000eb600000e35f00007d
:104b0800d75e0000c75d0000b35c00009c5b00003e
:104b1800825a000064590000425800001d570000e6
:104b2800f5550000c95400009b530000685200006e
:104b380033510000fb4f0000bf4e0000814d0000c4
:104b48003f4c0000fb4a0000b449000069480000df
:104b58001c470000cd4500007a44000025430000b2
:104b6800ce41000073400000173f0000b83d000030
:104b7800563c0000f23a00008c390000243800004e
:104b8800ba3600004d350000df3300006e320000f9
:104b9800fb300000872f0000112e0000992c000028
:104ba8001f2b0000a329000026280000a8260000cb
:104bb80028250000a6230000232200009f200000d3
:104bc8001a1f0000931d00000b1c0000821a000031
:104bd800f91800006e170000e215000055140000d7
:104be800c81200003a110000ab0f00001c0e0000b4
:104bf8008c0c0000fb0a00006a090000d9070000bd
:104c080048060000b60400002403000092010000da
:104c1800ff7f00000000000000000000000000000e
:104c2800000000000000000000000000000000007c
:020000040000fa
:104c3800f0874700889fbe008a9fbe008c9fbe00f9
:104c48008e1f7800d0b79f00e1b79f00f2b79f0092
:104c580083bf9f0004077800850678000000eb00fa
:104c6800c0b79f000300e00029003a003400370075
:104c78003c03be000dd0b900008045004200dd00b5
:104c8800efb09700010040001032b800100190000a
:104c980002b1b90005014100100078000780b90091
:104ca800800241000804420089844a000a05e8009d
:104cb8008a0f5700eeff3a002fb197000899be00ff
:104cc800a2b79f008b05e8008b8f56000a003200c0
:104cd8006044b8000e00e000f7ff3200bfb0970054
:104ce8004208dd005fb19700020640000005eb00b6
:104cf8006044b800deff37004fb097000000e800be
:104d0800c0b79f008fb89700808f50000c0032000a
:104d18000d00e000f8ff32004fb197000e90b90087
:104d2800b0b79f000d90b9004200dd00ffb09700ba
:104d380000804000a0b79f008005eb00e4ff37002b
:104d48004f0778004f06be004f05be004f04be0057
:104d58000f01b10000000600889fbe008a9fbe00b8
:104d6800800478000104780082037800049ab9006e
:104d7800040378000400e0000c0032000002eb009d
:104d880084017800078141008380440003004400c7
:104d98001105be003019450020914d000402e800bd
:104da800e4814100840f5300f6ff3a004f05be002e
:104db8004f04be0000000600889fbe0080047800f3
:104dc8000104780082037800049ab900040378008b
:104dd8000400e000100032000002eb0084017800bb
:104de80003814300038044001000be00880278005d
:104df8008502e900030033008180d1000080d300e0
:104e0800fbff37000089be000402e800e48141008e
:104e1800860f5200f2ff3a004f04be000000060061
:104e2800e4874700889fbe008a9fbe008c9fbe0013
:104e38008e1f780080bf9f000206be000107780021
:104e480005a2b900840578000400e0000d003200d6
:104e58000005eb008a047800090447008fb8970022
:104e6800098040000c01be001000be00d3ee070010
:104e7800008cbe000a05e800e48444008b0f55004e
:104e8800f5ff3a004f0778004f06be004f05be00f9
:104e98004f04be004f00b100000006001001be0024
:104ea8008288be0020019000b001900060011100ce
:104eb800e0811900a2009800b3009800400190001a
:104ec800d001900060011100e0811900c200980033
:104ed800d300980060019000f0019000600111007b
:104ee800e0811900e2009800f30098000000060035
:104ef800800278003501be008288be001501be0020
:104f080060011100e0811900a2009800b300980028
:104f1800680340001601be0060011100e08119001d
:104f2800c2009800d30098006c0240001401be0033
:104f380060011100e0811900e2009800f300980078
:104f48001501be0082089800930898001001be0061
:104f5800a2089800b30898001401be00600111006f
:104f6800e0811900c2089800d30898001601be0015
:104f7800e2089800f30898001601be008210980015
:104f8800931098001401be00a2109800b310980066
:104f98001001be00c2109800d31098001501be0081
:104fa80060011100e0811900e2109800f3109800e8
:104fb8001401be0082189800931898001601be00cc
:104fc80060011100e0811900a2189800b318980038
:104fd8001501be00c2189800d31898001001be0031
:104fe800e2189800f318980000000600ef02b000dd
:104ff800889fbe008a9fbe008c9fbe008e1f7800cf
:10500800010778001001be00b2b79f00c3b79f0028
:1050180020029000b002900094b79f00a5b79f00af
:1050280040039000d0039000f6af9f0087b79f0021
:1050380060049000f0049000d8af9f00e9af9f0093
:10504800bfb097000108b800b0af9f00c1af9f0084
:105058000390b90000004000cfa8970081004000ed
:10506800c1af9f009fb197000319b80092af9f008e
:10507800a3af9f0005a0b9000000400083014000d5
:10508800a3af9f00ffaa9700052ab800f4a79f00c6
:1050980085af9f0007b0b9000000400085024000be
:1050a80085af9f00dfab9700073bb800d6a79f00ee
:1050b800e7a79f0009c0b90000004000870340002f
:1050c800e7a79f001fac9700afac97007fa19700a0
:1050d8008fa9970008004100898049005fa29700c6
:1050e800efa2970004004000858048003fab97007e
:1050f800cfab97000600400087804800b0a79f000c
:10510800c1a79f00bfb497007fac9700084cb800b8
:10511800f8b79f0089bf9f00bfb497000fb59700ed
:105128000ac8b9000fbe97000c004000ffa89700fe
:105138004fb297000489b9000201400082bf9f0066
:105148009fb397005fab9700063bb800d6b79f00a8
:10515800e7b79f009fb397006fac970008b8b900f6
:10516800efb49700090040005fad97002fb6970095
:105178000cd1b90002014000e2b79f007fb0970050
:105188008fb897005fb29700efb297000001420016
:1051980081814a003fa39700cfa397008780d10061
:1051a8000680d300800f5100818f59000b00340016
:1051b800000feb0000002400100798003fb1970093
:1051c800cfb197005fa89700efa89700c612070015
:1051d80000004000200798008b0037006000100096
:1051e800e0801800800f5100818f59000c003d00ad
:1051f800000feb0000002c00100798003fb197004b
:10520800cfb197005fa89700efa89700b6120700e4
:105218000000ea0000004000200798007a003700ec
:105228001fac9700afac970060011400e0811c0030
:105238007fa097008fa89700000151008181590035
:105248005fa29700efa29700040141008581490001
:105258003fab9700cfab970006014100878149001b
:105268000c0024000d0020000201460083814e003e
:10527800c11bdd004f11de0002817300cf99de00f3
:105288003fb497009fb497000940b8002fb3970028
:1052980006c2b9000102420009047800cfb49700a1
:1052a80009c3b900860042007fad97005faa970046
:1052b8000453b800efac970009d2b90007024200c6
:1052c8005fad97008fb2970005d4b90088034200fc
:1052d8000000430081804b000a0022000b002000e0
:1052e8000000450081804d00420bdd004e00de00cd
:1052f80000007300ce88de007b120700000f7800e4
:105308007fb497008fbc97005fb19700efb197000b
:105318000200540083805c00020028000300200083
:105328003fa29700cfa29700040141008581490060
:105338004099de00cf91de00a0ed0700eb110700d9
:10534800100798001fab9700afab97007fa497009a
:105358008fac97000801530089815b005fa097001c
:10536800efa0970000015100818159003faa9700e2
:10537800cfaa970004014100858149000201460037
:1053880083814e00c11add004f11de0002817200d8
:10539800cf99de003fb39700dfab97000730b80026
:1053a800efac970009b2b90001024200cfb29700f2
:1053b80005bbb900860042001fb49700ffac9700f8
:1053c8000943b800080678000fb4970008e2b9004e
:1053d80007024200afb2970005ccb900880342002b
:1053e8000000430081804b000000450081804d0093
:1053f800420bdd004e00de0000007300ce88de00a8
:1054080039120700200798004f0778004f06be00a2
:105418004f05be004f04be00ef02b10000000600b9
:10542800ef0eb000889fbe008a9fbe008c9fbe0012
:105438008e1f7800f2af9f0083b79f0094b79f003c
:10544800a5b79f00110178006112b900f49f9f0071
:1054580085a79f00110190006113b90096a79f00ce
:10546800a7a79f00a10090006109b900b2a79f00fb
:10547800c3a79f001084d100900090008184d100c0
:10548800200090000085d1000800780077110700ff
:105498000006780008007800671107000007780008
:1054a80009007800711107000004780009007800ed
:1054b80061110700800578000a0078006b11070069
:1054c800800478000a0078005b1107000003780068
:1054d8006142b900d4a79f00e5a79f006160b900a9
:1054e800b0af9f00c1af9f00dfa09700000ab800cf
:1054f800cfa997000388b90005004000bfab97000b
:10550800efa0970001b9b90082024000c12bdd006d
:105518004f21de0002817300cfa9de00d29f9f00d9
:10552800e39f9f006148b90090af9f00a1af9f0023
:105538006159b900b29f9f00c39f9f006175b90070
:105548000a16b800bf9997000b98b9000d004000e3
:105558004f9a970004d1b90082064000c16add0065
:105568004f66de000c867200cfeede006130b900b7
:10557800f0a79f0081af9f00df9897001fa99700b1
:10558800020bb8002faa97000488b9000700400052
:10559800ef9897000191b900820340004139dd007e
:1055a8004f33de0006037100cfbbde007fa29700f9
:1055b8000461b8008faa970005e0b9000300400015
:1055c8000da2b90084014000411add004f11de0030
:1055d80002017200cf99de0006014100878149006f
:1055e800b2379f00c3379f00dfa297000a2cb8008c
:1055f8000ba8b90009004000efa3970007d1b90034
:10560800820440004148dd004f44de000804700079
:10561800cfccde00bfa897003f999700020db800d5
:105628004f9a97000488b9000b0040004fab9700d1
:105638000691b90082054000c15bdd004f55de00d0
:105648000a857300cfddde001fa897000a02b800a4
:105658000b80b900050040002fab970006d1b900b8
:1056680082024000c12bdd004f22de00048273005d
:10567800cfaade007fa097000801b8000980b90012
:10568800030040008fa8970001c3b90086014000bd
:10569800411bdd004f11de0002017300cf99de00cf
:1056a8000202520083825a00d4379f00e5379f00d8
:1056b8009fab9700083ab80009b8b9000500400048
:1056c800afa9970003c4b90088024000412bdd0050
:1056d8004f22de0004027300cfaade00ffa397006a
:1056e8000a39b800070378000bb8b9000300400076
:1056f8008fab970007d5b9008a0140004118dd003b
:105708004f11de0002017000cf99de000402410053
:1057180085824900f4379f00853f9f00df989700f6
:1057280006017800060ab8000788b900050040009d
:10573800ef9897000191b900820240004129dd00ed
:105748004f22de0004027100cfaade001fab9700d3
:105758000c31b8000db0b90003004000afa89700a5
:1057680001e6b9008c014000411bdd004f11de004d
:1057780002017300cf99de000202520083825a00b0
:10578800943f9f00a53f9f0061f02f008f8040004d
:105798001fb09700c1fd07006ef72f000f074700e5
:1057a8008e00780060f02f000f004000d0fd070049
:1057b80044002000840178000e01780021002000b8
:1057c8000e0078007cfd070068f22f000f044400eb
:1057d80015002000440020008401780008017800aa
:1057e80061f62f008f8040000e00780010fd070042
:1057f800140020004300200008017800d100200098
:10580800080078006cfd07006000b800b01f9f001a
:10581800c11f9f001804be007f9997008fa19700b1
:105828004718dd00c910de00810070004710dd0058
:105838002fb3970036025000a6825800b4b79f00d5
:10584800c5b79f005f1297000441b8006f1097001a
:1058580000c0b9000300400009a2b900840140005b
:105868000c0024000d0020000201460083814e0038
:10587800c11bdd004f11de0002817300cf99de00ed
:105888000fb09700400390000612b8005005900032
:105898000a90b9000500400003b1b9008202400037
:1058a8003fb19700cfb197000200420083804a00c1
:1058b800d01f9f00e11f9f001fa29700afa2970073
:1058c8004729dd00c921de00830171004721dd0081
:1058d800afb2970025009000b5009000000151007c
:1058e80081815900d2b79f00e3b79f007f129700cc
:1058f8000440b8000f19970002c1b9000101410026
:1059080009a2b900840041000000460081804e00d1
:10591800c10bdd004f00de0000807300cf88de0081
:105928000602b8000a81b9000501410001b0b900ba
:10593800800241005fb19700efb19700020042007a
:1059480083804a00f01f9f0081279f003fa2970095
:10595800cfa297004729dd00c921de00830171002d
:105968004721dd00afb2970045009000d5009000b8
:105978000001510081815900f2b79f0083bf9f0049
:105988001f1a97000440b8002f19970002c1b900e8
:105998000101410009a2b90084004100000046004d
:1059a80081804e00c10bdd004f00de0000807300d7
:1059b800cf88de000601b8000a85b9000305450056
:1059c80001b3b900860145007fb297008fba9700ee
:1059d800040041008580490090279f00a1279f006f
:1059e8008e0078001fb0970041fd0700440020009a
:1059f800840178000e017800510020000e00780024
:105a0800edfc0700140020004300200062f32f0083
:105a18000f0141005100200002007800e6fc070059
:105a280069f42f008f8444001500200044002000f2
:105a3800840178000901780061f32f008f8040000d
:105a48000e0078007afc070068f52f000f04440068
:105a580014002000430020000801780061002000a5
:105a680009007800d4fc07008fb297002511900038
:105a7800b51190001500200044002000880078002f
:105a880008007800e6fc070014002000430020000e
:105a980062f32f000f0141009fb0970008007800c3
:105aa800adfc07003f1d9700cf1d97000a53b800b3
:105ab800d6af9f00e7af9f000bd0b90000004000b1
:105ac80087034000e7af9f005f199700ef19970021
:105ad8007f1a97008f2297001f239700af23970004
:105ae8005fa89700efa897000004460081844e0045
:105af800c148dd004f44de0008847000cfccde00d2
:105b08000210b8000391b900020141008100410070
:105b18000000460081804e004109dd004f00de0094
:105b280000007100cf88de00080440008984480026
:105b38000420b80005a2b900040242008100420016
:105b48000000460081804e00c109dd004f00de00e4
:105b580000807100cf88de00080440008984480076
:105b68000630b80007b3b9000603430081004300bc
:105b78000000460081804e00410add004f00de0033
:105b880000007200cf88de000804400089844800c5
:105b98008984d1000884d30000002d00f1ff2f0074
:105ba800080040008980480005002200850f500049
:105bb800e08f5800540036000801be005fa8970027
:105bc800efa897007deb0700b50f07000000d10094
:105bd8006101b8001fb39700028bbe003f18970001
:105be800cf189700e00f5000e08f580003003d00e9
:105bf80060001100e0801900008bbe009fb3970081
:105c0800648543005f199700ef1997000210b800e8
:105c18000391b90002014100810041000801be0062
:105c280066eb07009e0f07000000d1006101b80075
:105c3800028dbe005f189700ef189700e00f500024
:105c4800e08f580003003d0060001100e08019005b
:105c5800008dbe001fb09700680540007f199700af
:105c68008f2197000210b8000391b900020141008a
:105c7800810041000801be0050eb0700880f0700b3
:105c88000000d1006101b800028dbe007f189700a6
:105c98008f209700e00f5000e08f580003003d0070
:105ca80060001100e0801900008dbe009fb09700d1
:105cb8006c8540001f219700af2197000210b800a3
:105cc8000391b90002014100810041000801be00b2
:105cd8003aeb0700720f07000000d1006101b8001d
:105ce800028dbe001f209700af209700e00f5000e4
:105cf800e08f580015003d0060001100e080190099
:105d0800008dbe00110037001fb197000a89be0040
:105d18005f1a9700ef1a97001fb3970024039800a3
:105d2800350398007f1897008f2097001fb19700c0
:105d380040019800510198001f229700af22970058
:105d48001fb397006403980075039800ffa8970095
:105d580060f32f000f004000a4fc07003f149700d9
:105d6800cf14970067f12f000f8643000fb09700fc
:105d780060039000f003900060031300e0831b00b1
:105d88005f1297000440b8006f11970002c1b90074
:105d98000101410009a2b900840041000a00240061
:105da8000b0020000000450081804d004109dd0006
:105db8004f00de0000007100cf88de000032b8001e
:105dc80001b1b900050141000780b9008002410016
:105dd800048ebe007f1297000440b8000f19970088
:105de80002c1b9000101410009a2b90084004100c3
:105df8000000450081804d00c109dd004f00de0034
:105e080000807100cf88de000032b80001b1b9000f
:105e1800050141000780b90080024100d40f9f00ae
:105e2800e50f9f001f1a97000440b8002f1997002c
:105e380002c1b9000101410009a2b9008400410072
:105e48000000450081804d00410add004f00de0062
:105e580000007200cf88de000032b80001b1b9003e
:105e6800050141000780b90080024100f40f9f003e
:105e780085179f0025f22f000f8142001c00be00ed
:105e8800450bdd00cb00de00810073004500dd001e
:105e9800009ebe008c0f5100f8ff3a0068f32f00f7
:105ea8000f0444008fb3970027119000b71190009a
:105eb80015002000340020008800780066f12f00cb
:105ec8000f004300d6fb0700140020003300200019
:105ed8002fb1970082007800080078009efb070029
:105ee8004f0778004f06be004f05be004f04be00a6
:105ef800ef0eb100000006006f06b000889fbe00dc
:105f08008a9fbe008c9fbe008e1f7800d2b79f006c
:105f1800e3b79f00f4b79f0085bf9f001101780089
:105f28006112b900b4a79f00c5a79f001101900096
:105f38006113b900d6a79f00e7a79f00a1009000b2
:105f4800610cb900f8a79f0089af9f00100290006c
:105f5800cfa2de0020019000cf91de001000780073
:105f6800cf80de00d08f9f00e18f9f00f48f9f00cd
:105f780085979f0092979f00a3979f0068fb2f002b
:105f88000f044400880078007fb09700c3fb070027
:105f98001800be0090b79f00a1b79f001fa49700ec
:105fa800afa4970000054000818548005f9a9700dc
:105fb800ef9a97000401420085814a000242b80026
:105fc80003c0b900050040000991b90082024000f1
:105fd80006002400070020000402430085824b00cd
:105fe800c12bdd004f22de0004827300cfaade0041
:105ff8007f9f97000a70b8000bf1b90001014100ba
:106008000fa797000ed3b9008600410002002400b4
:10601800030020000000410081804900c109dd0023
:106028004f00de0000807100cf88de0004024000cf
:10603800858248001e0028000e26b80004815600fc
:106048000ea8b900800641000400240005002000c5
:106058000c0642008d864a00c16add004f66de00ec
:106068000c867200cfeede007f9b97008fa397000f
:106078000601430087814b000242b80003c0b90003
:10608800050040000991b900820240000000240088
:10609800010020000402400085824800c128dd007c
:1060a8004f22de0004827000cfaade005f999700bd
:1060b8000a10b8000b91b90001014100ef9b97004d
:1060c80007d5b9008a00410002002400030020001f
:1060d8000000410081804900c109dd004f00de0059
:1060e80000807100cf88de000002520081825a00d1
:1060f8000e25b800048155000ea8b900800541009e
:1061080004002400050020000a0542008b854a008f
:10611800c15add004f55de000a857200cfddde0072
:106128000843b80009c4b9000804440087034400c0
:1061380008002400090020000603440087834c005f
:10614800c13cdd004f33de0006837400cfbbde00a8
:106158001fb097000001b800afb297000580b900e2
:1061680000004000830140000800240009002000ce
:106178000201440083814c00c11cdd004f11de0088
:1061880002817400cf99de005f9a97000420b8005e
:10619800ef9c970009a2b900040242008100420066
:1061a80004002400050020000000420081804a000d
:1061b800c10add004f00de0000807200cf88de00db
:1061c80000015100818159007f9c97000840b80068
:1061d800880478000fa4970008cab9000402420096
:1061e8008100420004002400050020000000420055
:1061f80081804a00c10add004f00de000080720085
:10620800cf88de000001510081815900060341005a
:10621800878349000e32b800068052000eb9b900d3
:106228008202400006002400070020000402430008
:1062380085824b00c12bdd004f22de0004827300f3
:10624800cfaade005fa497000441b80005c0b900da
:10625800030040006fa797000ea3b9008601400015
:106268007fa097000a03b8000b80b9000700400020
:106278000faf97000ed4b900880340000601510003
:106288008781590070014100e08149004b18dd0009
:106298004511de0002017000c599de00f2879f00fb
:1062a800838f9f00ffa097000c09b8000d88b900e4
:1062b800030040000ee3b90086014000bfa4970028
:1062c800044bb80005c8b90007004000cfa09700ec
:1062d80001a2b900840340000601510087815900da
:1062e80070014100e08149004b1add004511de00d4
:1062f80002017200c599de00928f9f00a38f9f0054
:106308000a49b8000bc8b90003004000cfa39700a2
:1063180007d5b9008a0140005fa497000c42b80075
:106328000dc0b900050040006fa797000ee6b90040
:106338008c02400004015100858159007001410020
:10634800e08149004b18dd004511de0002017000b4
:10635800c599de00b28f9f00c38f9f006000b80010
:10636800b0979f00c1979f006fb59700ca02b00011
:106378000006eb00a1fa2f008f854000e2f82f00fd
:106388000f0141000c00410060019000f0019000f5
:10639800421add00ce11de00830172004211dd00d9
:1063a8008fba97000c8242000000220001002000f2
:1063b80034034000a48348000600be00c20bdd0081
:1063c8004e00de0000807300ce88de000001510020
:1063d800818159006fb49700680b90000612b800cd
:1063e800780890000090b9000500400003b3b90098
:1063f800860240000408b0000580b000c82cdd000b
:106408004822de0004827400c8aade003a00420076
:10641800aa804a000002be00008dbe00e1f82f00ed
:106428008f8040008c814000480b90001330b800ea
:106438001301900002b3b90001034300130178006f
:10644800efb19700530c90000891b9008200430007
:106458000008b0000180b000480bdd004800de00f5
:1064680000007300c888de000402400085824800ee
:10647800000028000100200004004000858048003a
:106488004088de00cf80de00809dbe00c000dd00b9
:10649800000020000002520081825a00049dbe00c4
:1064a80064064600ec0f5600b4ff3a00ffb49700ac
:1064b8001904be00f8af9f0089b79f00ffb097008e
:1064c80021009000b1009000d0af9f00e1af9f0085
:1064d800ffb1970043019000d3019000b2af9f0035
:1064e800c3af9f00ffb2970065029000f5029000cd
:1064f80094af9f00a5af9f001f9d9700af9d970089
:106508007fab9700bf9397000734b8004f9197006f
:1065180002b0b900090040008fb2970005b9b90070
:10652800820440000c0024000d00200008044600ee
:1065380089844e00414bdd004f44de00080473009f
:10654800cfccde005faf97005f9097000073b80074
:10655800ef91970003f0b900070040005f929700a1
:10656800efaa970005a1b900820340000603460080
:1065780087834e00413fdd004f33de00060377007e
:10658800cfbbde003fa99700ff9197000310b8002a
:106598008f9a97000591b900010141007f979700f4
:1065a800cfa9970003f2b90084004100000046001b
:1065b80081804e00410add004f00de0000007200bd
:1065c800cf88de0006034000878348009faa970013
:1065d8000a28b8000ba9b90001014100afa997002a
:1065e80003d2b900840041000000460081804e00bb
:1065f800410add004f00de0000007200cf88de0097
:1066080006034000878348000604540087845c0022
:106618007fb797008e027800351f4400259f4c00f5
:106628007fac9700df9497000943b800ef9197007b
:1066380003c0b900070040008fb2970005c9b90030
:10664800820340000603460087834e00413cdd007c
:106658004f33de0006037400cfbbde00bf94970003
:106668005fa997000248b800efaa970005c9b900ca
:10667800010141005fac9700cf94970009c2b900af
:10668800840041000000460081804e004109dd0081
:106698004f00de0000007100cf88de0006034000d6
:1066a80087834800bfa997000a18b8000b99b9005a
:1066b800010141004fac970008d2b90084004100a5
:1066c8000000460081804e00c10cdd004f00de0056
:1066d80000807400cf88de000603400087834800ee
:1066e8007f9197009fa997000310b800afaa970061
:1066f8000591b900010141001fac97008f9c9700dc
:1067080009c2b900840041000000460081804e00a3
:106718004109dd004f00de0000007100cf88de0077
:106728000003530081835b001e0f43005e974b00fc
:10673800ffb19700e8814100c3b79f007faa970087
:10674800ff9297000523b8008f9c970009a0b90015
:10675800070040000fb2970004a9b9008203400067
:106768000603460087834e00c13add004f33de0042
:1067780006837200cfbbde003f949700bfac970042
:106788000940b800cfaa970005c1b900010141002e
:1067980009047800cf94970009c2b9008400410029
:1067a8000000460081804e004109dd004f00de00f8
:1067b80000007100cf88de00060340008783480090
:1067c800df9197001faa97000418b8002fac970014
:1067d8000899b90001014100ef91970003a2b9009f
:1067e800840041000000460081804e00410add001f
:1067f8004f00de0000007200cf88de000603400074
:1068080087834800dfaa97000a28b8000ba9b900b7
:1068180001014100efac970009d2b90084004100a2
:106828000000460081804e004109dd004f00de0077
:1068380000007100cf88de000003530081835b00f5
:10684800cfb1970093094300d3914b007fb29700d3
:106858006c024200b4b79f007fab97000a32b800c1
:106868000bb0b900050040000fb4970008d5b90077
:106878008a0240000402460085824e00c12cdd00d9
:106888004f22de0004827400cfaade003f919700f9
:106898009fa997000310b800afab97000791b90004
:1068a800010141001fac9700cf94970009c3b900bc
:1068b800860041000000460081804e004109dd004d
:1068c8004f00de0000007100cf88de0004024000a7
:1068d80085824800dfa997007f9397000618b800c3
:1068e8000f9c97000899b90001014100efa9970092
:1068f80003b3b900860041000000460081804e00c5
:10690800410bdd004f00de0000007300cf88de0081
:106918000402400085824800df9397003fac97004f
:106928000838b8004fab970006b9b900010141001b
:10693800ef94970009c3b9008600410000004600a3
:1069480081804e004109dd004f00de00000071002b
:10695800cf88de000002520081825a003fb49700bf
:1069680038034200a8834a000602be00068cbe0017
:10697800ffb497001905be001e01be004fb0970076
:106988001003be000a54b8000bd0b9000000400044
:10699800890440000210b8000391b90002014100c7
:1069a8008100410008044000898448000421b8009f
:1069b80005a2b90004024200830142000630b80073
:1069c80007b3b900060343008100430002014000f9
:1069d8008381480008044100898449000400280094
:1069e800f5ff23000802520089825a0040aade00ff
:1069f800cfa2de000450b80005d1b9000101410062
:106a08000ba3b900860041000000460081804e00bb
:106a18004109dd004f00de0000007100cf88de0074
:106a2800ffb197008019450081914d001e04be00fa
:106a38000820b80009a1b9000101410005c3b90047
:106a4800860041000000460081804e00410bdd00b9
:106a58004f00de0000007300cf88de00001f4400f6
:106a680001974c00cfb397001704be000820b80068
:106a780009a1b9000101410005c3b9008600410020
:106a88000000460081804e00410fdd004f00de000f
:106a980000007700cf88de004fb19700001944004e
:106aa80001914c00bfb197001303be000620b80047
:106ab80007a1b9000101410005b2b90084004100f5
:106ac8000000460081804e00410add004f00de00d4
:106ad80000007200cf88de00bfb29700801a430022
:106ae80081924b000004eb000a0020001b002000ec
:106af8000fbb970086034400e9f82f008f844400f9
:106b0800888144006fb797000e1290001320b800d8
:106b18001301900002a2b90001024200130178009b
:106b28001e1390000691b900820042000000450043
:106b380081804d004188de00cf80de00971b100069
:106b48009793180064044400ec0f5400e8ff3a00df
:106b5800dfb097007fb0970024f907004f0778004f
:106b68004f06be004f05be004f04be006f06b100c1
:106b78000000060011002000010878008000eb00ea
:106b8800110098002100980031009800410620006b
:106b980041009800810b2000510098000000060079
:106ba80000027800830078001300e000060032003d
:106bb8000000e000040034000000eb0080097800c9
:106bc800a40198009001980000802000800f5200d6
:106bd80001003400210290002100900004015000bf
:106be8008201780001003b008201ea004100900028
:106bf800808f510003003400110090000000410014
:106c0800900098001100900000004200b000980029
:106c180051009000800f520003003c000000eb0080
:106c280090009800b4009800a400980000000600a6
:020000040000fa
:106c3800889fbe008a1f78008004eb00882f2100ff
:106c480008844400a02021000080440002002000a5
:106c5800036824001000be0074e60700020020004c
:106c680003f02300ace6070008e70700008cbe002d
:106c78008833210008844400a024210000804400b7
:106c8800529f2000633324001000be0067e607000f
:106c98000200200003f023009fe60700fbe6070040
:106ca800008cbe008837210008844400c0282100d9
:106cb8000080440002002000036824001000be0089
:106cc8005ae607000200200003f0230092e60700be
:106cd800eee60700008cbe00e484440000042000b7
:106ce800808f5400d5ff3a006000b800209b8800d0
:106cf800319b8800a09a8800b19a8800209a880061
:106d0800319a88008004eb008a3b2100c02c2100c6
:106d1800008044000200200003f023001000be00a1
:106d28007de60700d9e60700001d7800083c210031
:106d380008844400c02d2100008044000200200087
:106d4800034824001000be0038e6070002002000b7
:106d580003f0230070e60700cce60700008cbe00b5
:106d6800e4844400ec8f5400e8ff3a00020020005d
:106d780003d8240020978000319780002be6070075
:106d88000200200003f0230063e60700bfe60700c7
:106d9800409e8800519e8800529f20006333240043
:106da800a0968000b196800020e60700020020002f
:106db80003f0230058e60700b4e60700e09d8800ca
:106dc8000200200003f02300c0968000d1968000c6
:106dd80051e60700ade60700f09d88008004eb004f
:106de800c83c210008844400802e21000080440013
:106df8000200200003f023001000be0046e6070052
:106e0800a2e60700008cbe00483d2100088444002b
:106e1800002f2100008044000200200003202400ed
:106e28001000be0001e607000200200003f0230066
:106e380039e6070095e60700008cbe00e4844400ac
:106e4800e88f5400e6ff3a000000eb004f05780099
:106e58004f04be0000000600ea874700889fbe0076
:106e68008a9fbe008c9fbe008e1f780001077800a5
:106e780010047800cfc4de0010059000cfd5de00e6
:106e880020069000cfe6de00c29780000243b800db
:106e9800d097800000c0b900070040000991b900f0
:106ea80082034000e29780000252b800f097800009
:106eb80000d0b900050040000b91b90082024000e3
:106ec8000603420087834a00029880000262b800e5
:106ed8001098800000e0b900050040000d91b9004d
:106ee800820240000603420087834a0020988000ff
:106ef8003198800006034000878348004739dd0049
:106f08004930de0000007100c9b8de00d0b79f002c
:106f1800e1b79f00429880000243b8005098800073
:106f280000c0b900070040000991b9008203400081
:106f3800629880000252b8007098800000d0b900b2
:106f4800050040000b91b900820240000603420090
:106f580087834a00829880000262b8009098800077
:106f680000e0b900050040000d91b9008202400020
:106f78000603420087834a00a0988000b1988000e9
:106f880006034000878348004738dd004932de00a9
:106f980004027000c9bade00f4b79f0085bf9f00e5
:106fa800c29880000243b800d098800000c0b900a1
:106fb800070040000991b90082034000e298800070
:106fc8000252b800f098800000d0b90005004000d7
:106fd8000b91b900820240000603420087834a00f1
:106fe800029980000262b8001099800000e0b900a0
:106ff800050040000d91b9008202400006034200de
:1070080087834a0020998000319980000603400058
:1070180087834800c738dd004931de0002817000ef
:10702800c9b9de0010002800f1ff2f005fb29700f9
:10703800efb29700800f5200818f5a0003003d0085
:1070480010002800000f78000b0037005fb0970091
:10705800efb09700f4ff2700840f5000e08f58002e
:1070680003003400f0ff2700000f7800020037000b
:10707800dfb29700050f780010002800f1ff2f00fd
:107088007fb297008fba9700800f5200818f5a0005
:1070980003003d0010002800100798000b0037007f
:1070a8007fb097008fb89700f4ff2700840f500037
:1070b800e08f580003003400f0ff27001007980005
:1070c80002003700ffb2970015079800100028004b
:1070d800f1ff2f00800f5100818f590003003d0000
:1070e800100028002007980008003700f0ff27004c
:1070f800800f5100e08f590003003400f0ff270093
:107108002007980001003700220798000000eb00d4
:107118004f0778004f06be004f05be004f04be0063
:10712800af00b10000000600ea874700889fbe0054
:107138008a9fbe008c9fbe008e1f780001077800d2
:1071480010047800cfc4de0010059000cfd5de0013
:1071580020069000cfe6de00c29980000243b80006
:10716800d099800000c0b900070040000991b9001b
:1071780082034000e29980000252b800f099800032
:1071880000d0b900050040000b91b9008202400010
:107198000603420087834a00029a80000262b80010
:1071a800109a800000e0b900050040000d91b90078
:1071b800820240000603420087834a00209a80002a
:1071c800319a800006034000878348004e39dd006d
:1071d8004230de0000007100c2b8de00d0b79f0068
:1071e800e1b79f00429a80000243b800509a80009d
:1071f80000c0b900070040000991b90082034000af
:10720800629a80000252b800709a800000d0b900db
:10721800050040000b91b9008202400006034200bd
:1072280087834a00829a80000262b800909a8000a0
:1072380000e0b900050040000d91b900820240004d
:107248000603420087834a00a09a8000b19a800012
:1072580006034000878348004e38dd004232de00d6
:1072680004027000c2bade00f4b79f0085bf9f0019
:10727800c29a80000243b800d09a800000c0b900ca
:10728800070040000991b90082034000e29a80009b
:107298000252b800f09a800000d0b9000500400002
:1072a8000b91b900820240000603420087834a001e
:1072b800029b80000262b800109b800000e0b900c9
:1072c800050040000d91b90082024000060342000b
:1072d80087834a00209b8000319b80000603400082
:1072e80087834800ce38dd004231de00028170001d
:1072f800c2b9de0010002800f1ff2f005fb297002e
:10730800efb29700800f5200818f5a0003003d00b2
:1073180010002800000f78000b0037005fb09700be
:10732800efb09700f4ff2700840f5000e08f58005b
:1073380003003400f0ff2700000f78000200370038
:10734800dfb29700050f780010002800f1ff2f002a
:107358007fb297008fba9700800f5200818f5a0032
:1073680003003d0010002800100798000b003700ac
:107378007fb097008fb89700f4ff2700840f500064
:10738800e08f580003003400f0ff27001007980032
:1073980002003700ffb29700150798001000280078
:1073a800f1ff2f00800f5100818f590003003d002d
:1073b800100028002007980008003700f0ff270079
:1073c800800f5100e08f590003003400f0ff2700c0
:1073d8002007980001003700220798000000eb0002
:1073e8004f0778004f06be004f05be004f04be0091
:1073f800af00b10000000600f6874700889fbe0076
:107408008a9fbe008c9fbe008e1f780001077800ff
:1074180010037800cfb3de0010069000cfe6de0040
:10742800200090006101b900f2b79f0083bf9f0060
:10743800c29b80000235b800d09b800000b0b90024
:107448000b0040000791b90082054000e29b8000d4
:107458000262b800f09b800000e0b900050040001f
:107468000d91b900820240000a0542008b854a004e
:10747800029c8000ffb19700021ab800109c80009f
:107488000098b900050040008fb897000191b90035
:10749800820240000a0542008b854a00209c800039
:1074a800319c80000a0540008b854800475add0062
:1074b8004951de0002017200c9d9de00f2af9f0017
:1074c80083b79f00429c80000234b800509c800023
:1074d80000b0b900090040000791b90082044000db
:1074e800629c80000262b800709c800000e0b900d5
:1074f800050040000d91b9008202400008044200d6
:1075080089844a00829c80007fb097000202b800fc
:10751800909c8000ffb197000098b90005004000da
:107528008fb897000191b900820240000804420018
:1075380089844a00a09c8000b19c80000804400017
:1075480089844800474add004941de000201720093
:10755800c9c9de0092b79f00a3b79f00c49c8000f2
:107568000431b800d09c800000b0b900030040008e
:1075780007a2b90084014000e49c80000463b800bd
:10758800f09c800000e0b900070040000da2b9009f
:10759800840340000201430083814b00049d800066
:1075a800ffb29700042bb800109d800000a8b90016
:1075b800070040008fb8970001a2b900840340007b
:1075c8000201430083814b00209d8000319d800093
:1075d8000201400083814800c99ade004718dd0097
:1075e8004912de0004027000b4b79f00c5b79f00bf
:1075f800c258dd004e55de000a857000ceddde0083
:107608000a50b8000bd5b9000a05450081004500ad
:10761800424add004e44de0008047200ceccde0093
:107628000845b80009c4b900080444008b054400a3
:10763800c21add004e11de0002817200ce99de0012
:107648000214b8000391b900020141008904410005
:107658000001450081814d000201440083814c00f6
:10766800409ede00cfe6de000c01be00d3e407003a
:107678000b090700010020007fa997008fb1970030
:10768800e00f5100e08f590007003c008180d100d5
:107698000080d30060001000e0801800d0b79f0081
:1076a800e1b79f00040037008180d1000080d3003b
:1076b800d0b79f00e1b79f000c01be000a00be00d2
:1076c800bee40700f6080700010020001fb297007b
:1076d800afb29700e00f5200e08f5a0005003c005f
:1076e8008180d1000080d30060051000e08518007b
:1076f800020037008185d1000085d3000c01be004f
:107708000800be00ade40700e508070001002000fe
:107718003fb19700cfb19700e00f5100e08f5900bb
:1077280005003c008180d1000080d300600110007a
:10773800e0811800020037008181d1000081d30068
:1077480010002800f1ff2f005fb29700efb29700fa
:10775800800f5200818f5a0003003d00100028005e
:10776800000f78000b0037005fb09700efb097006c
:10777800f4ff2700840f5000e08f58000300340006
:10778800f0ff2700000f780002003700dfb29700f3
:10779800050f780010002800f1ff2f00800f55001a
:1077a800818f5d0003003d0010002800100798003d
:1077b80008003700f0ff2700800f5500e08f5d00bc
:1077c80003003400f0ff270010079800010037007d
:1077d8001a07980010002800f1ff2f00800f5100b1
:1077e800818f590003003d001000280020079800f1
:1077f80008003700f1ff2700810f5100e08f590082
:1078080003003400f0ff270020079800010037002c
:1078180022079800509480000000cf000000e90083
:107828004f80de004f0778004f06be004f05be00b0
:107838004f04be006f01b10000000600881f7800e9
:1078480001047800813b210010017800910051006b
:1078580010009000d29d800002005000e008070050
:10786800cf80de00be13e20002003d008000ea0087
:107878000100370080007800e09d8000008c400007
:107888000000eb004f04780000000600f287470074
:10789800889fbe008a9fbe008c9fbe008e1f780006
:1078a80000057800e2b79f00800578003b02780069
:1078b800cfa2de001b037800cfb3de0064074000d0
:1078c8001e047800cfc4de00110078006101b90001
:1078d80092b79f00a3b79f00110090006101b90003
:1078e800b2b79f00c3b79f00210090006106b9009e
:1078f8000421b80005a2b900040242008301420035
:107908004a18dd00c610de00810070004a10dd0054
:107918000632b80007b3b9000603430085024300e6
:107928000201420083814a000842b80009c4b90034
:1079380008044400850244000201420083814a0091
:107948004a1add004611de0002017200c699de0007
:107958001ae40700720807001a00e00004003d005e
:107968000000ea006fb39700100398000200370088
:10797800efb09700900098009e00ea001b00ea0014
:10798800970807006fb49700001c7800180078006b
:107998003608070000077800180078002608070056
:1079a800d0b79f006fb19700120078002f0807002a
:1079b80000057800efb19700130078001e08070053
:1079c8006104b900cfd5de006171b9001fb397001b
:1079d8000232b80003b0b90005004000afb097000c
:1079e8000191b90082024000412bdd004f21de00e9
:1079f80002017300cfa9de00f2b79f0083bf9f008a
:107a08003fb097000803b8000980b900070040009c
:107a18004fb2970004c1b900820340004138dd002d
:107a28004f33de0006037000cfbbde000a61b800ea
:107a38000be0b900030040000dd2b90084014000fa
:107a4800c118dd004f11de0002817000cf99de0001
:107a580006034100878349005fb197006112b900ae
:107a68000431b80005b0b9000300400007a2b9000e
:107a780084014000411add004f11de00020172004e
:107a8800cf99de007fb39700020743000861b80072
:107a980009e0b900030040000dc2b90084014000ac
:107aa800cf9bde004118dd004f13de000603700097
:107ab800bfb097000a09b8000b88b900030040005e
:107ac800cfb0970001d2b90084014000411add000f
:107ad8004f11de0002017200cf99de000200530050
:107ae8008e0078003e0807006fb3970020039800c7
:107af8000000eb004f0778004f06be004f05be00a0
:107b08004f04be002f01b10000000600f8874700af
:107b1800889fbe008a9fbe008c9fbe008e1f780083
:107b28008005780082067800030778000005780051
:107b38003a027800cfa2de001a017800cf91de0069
:107b4800640640001c037800cfb3de001100780003
:107b58006104b900a8b79f00b9b79f001100900051
:107b68006104b900c8b79f00d9b79f000214b800d4
:107b78000391b90002014100890441004a48dd002f
:107b8800c640de00810070004a40dd000421b800d4
:107b980005a2b90004024200830142000201440028
:107ba80083814c000632b80007b3b90006034300ce
:107bb800850243000201420083814a00ca1cdd009d
:107bc8004611de0002817400c699de007be30700df
:107bd800e20707001a00e00002003d00000fea007b
:107be80001003700000f78000e84e8009c00ea00ce
:107bf8001b00ea00fa070700000c78001e00780056
:107c08009a07070080bf9f001e0078008a070700b8
:107c1800000678001800780094070700000578002f
:107c280018007800840707001d04be008fb897006d
:107c3800610ab9000823b80009a1b9000701410089
:107c480005c2b90084034100413add004f31de002e
:107c580002017200cfb9de00e2af9f00f3af9f00d0
:107c680000e1b9004f91de006112b9000443b80089
:107c780005c1b9000701410009a2b9008403410008
:107c8800413add004f31de0002017200cfb9de005b
:107c980082b79f0093b79f006153b9000642b800ae
:107ca80007c1b9000501410009b3b90086024100c6
:107cb80060021200e0821a00cfadde00412cdd0028
:107cc8004f25de000a0574002d049000bd049000c5
:107cd8006163b9000832b80009b1b9000501410073
:107ce80007c3b90086024100c128dd004f22de002b
:107cf80004827000cfaade002fb19700bfb19700b1
:107d08000206420083864a008fb997000098b9009e
:107d18004f80de006101b9000242b80003c0b9001b
:107d2800050040000991b90082024000412cdd00a5
:107d38004f22de0004027400cfaade004fb0970085
:107d4800dfb097000404500085845800efa897001e
:107d58000a09b8000b88b90003004000ffa8970083
:107d680001d2b90084014000411add004f10de0045
:107d780000007200cf98de00e0b79f00f1b79f00c7
:107d8800e00f5000e08f580003003a00f0ff230096
:107d9800200798002c0037000c51b8000dd0b9000e
:107da800030040000be2b90084014000cf9dde00d3
:107db8004118dd004f15de000a0570000fb097006e
:107dc8009fb0970060011000e08118000263b800be
:107dd80003e0b900070040000d91b900820340009c
:107de800efa897000809b8000988b9000300400007
:107df800ffa8970001c2b9008401400006034100b2
:107e080087834900413add004f31de0002017200ec
:107e1800cfb9de006fb49700ffb49700e00f5400ad
:107e2800e08f5c0004003d0060051500e0851d0042
:107e380060011100e08119008a00780002007800d2
:107e480067070700200798000000eb004f0778003d
:107e58004f06be004f05be004f04be008f01b100a3
:107e6800000006006102b80004007800c013bc00de
:107e7800209e8000000141008208780000802100d7
:107e8800800f510001003600800878000000eb00e8
:107e980000000600889fbe00010378006102b80058
:107ea80004007800c813bc000204be00529e800083
:107eb80002a1b900828444004248de00010020008b
:107ec800000b780002802100800f51000100310072
:107ed800020b78000000eb004f04be000000060013
:107ee8006102b80004007800cc13bc00809e8000ba
:107ef80000014100820878000000eb000000060045
:107f08006102b80004007800d413bc00c09e800051
:107f180000014100820878000000eb000000060024
:107f2800889fbe000004be0010007800cf80de00ed
:107f380077e207000200200043332400bbe107007a
:107f48000200200003802300b8e10700808cbe00f7
:107f580018009000cf80de006de2070002002000cc
:107f680043332400b1e1070002002000038023000e
:107f7800aee10700a0049800b10498002800900022
:107f8800cf80de0062e207000200200043332400b5
:107f9800a6e107000200200003802300a3e10700f8
:107fa800c0049800d10498004f04be0000000600e9
:107fb800889fbe000004be0010007800cf80de005d
:107fc80053e207000200200003d0230097e10700d6
:107fd800808cbe0018009000cf80de004ce20700c5
:107fe8000200200003d0230090e10700a0049800bd
:107ff800b104980028009000cf80de0044e207001a
:108008000200200003d0230088e10700c004980084
:10801800d10498004f04be0000000600889fbe00ef
:108028000004be0010007800cf80de0038e20700b0
:1080380002002000433324007ce1070002002000f6
:108048000390230079e10700808cbe00180090009f
:10805800cf80de002ee20700020020004333240018
:1080680072e1070002002000039023006fe107007f
:10807800a0049800b104980028009000cf80de008a
:1080880023e20700020020004333240067e10700d1
:10809800020020000390230064e10700c004980058
:1080a800d10498004f04be0000000600889fbe005f
:1080b8000004be0010007800cf80de0014e2070044
:1080c800020020000380230058e10700808cbe00d6
:1080d80018009000cf80de000de2070002002000ab
:1080e8000380230051e10700a0049800b104980020
:1080f80028009000cf80de0005e207000200200083
:108108000380230049e10700c0049800d1049800c7
:108118004f04be0000000600889fbe00810478005e
:10812800100478006140b900f9e107000800e00098
:1081380003003d00020020000378240076e10700d8
:108148000200200003a8230038e10700808cbe004d
:108158004f04be0000000600889fbe00810478001e
:10816800100478006140b900e9e107000800e00068
:1081780003003d00020020000378240066e10700a8
:0c818800808cbe004f04be00000006000a
:020000040000fa
:108194000f24b000889fbe008a9fbe008c9fbe0043
:1081a4008e1f7800c1602a0042db2f000f014100be
:1081b4007200410007000900311878000001b10085
:1081c4000101b1006000b800b0af9d00c1af9d00d7
:1081d400d0af9d00e1af9d00f0af9d0081b79d0041
:1081e4000004eb0098b79d00a8b79d00b8b79d00a8
:1081f400ca22a900020078000017b0005efa070046
:108204008cfa070080de2f000f004000c302070035
:1082140044c7bf0001ceb300014060003040b3004a
:1082240044e7b700303a800001e02f00010060000d
:10823400e000b300303a880044c7bf00f043b20006
:108244000064a00044e7b700150a0700460c0700c5
:108254002d0c0700d662a8008c0b0700ad0b07009d
:108264007b0b07008c0907000805070002090700bb
:1082740009070700bc07070000482800e1012000a7
:10828400490c0700d662a900e887880029de2f0080
:108294008f84440068004400f10b07008800440008
:1082a40080b07c00e88780000804e800e887880044
:1082b400e20f5400f7ff34006000b800801f9f00f5
:1082c400911f9f00a01f9f00b11f9f00c01f9f0010
:1082d400d11f9f00e01f9f00f11f9f0080279f0078
:1082e40091279f00a0279f00b1279f00c0279f00d0
:1082f400d1279f00e0279f00f1279f0060ec2f000b
:10830400f1ff2f00802f9f00912f9f00c35d20005d
:10831400f3b79f001d0020000007eb0001003700a9
:108324008006eb00e613e200feff3200ee878800d1
:108334000e0078000af62f000f054500abf52f005c
:108344008f85450068004000c50b070000017800d8
:10835400e08780000000400021de2f008f80400075
:10836400e08078008100510001307d0064404000cd
:10837400bc0a070080447800e887800008044400b1
:1083840065404400b70a07008980fb004800dd000f
:108394000080400000b47d00fc10ec00e087880001
:1083a400e20f5000e7ff3400f0002000ac0b0700a0
:1083b4000006780041f52f008f8040000b00780004
:1083c400a6fa070081f62f008f8040000a0078008b
:1083d40056fb0700ee878800869f8000979f8000e9
:1083e4000e0078008e02780008f32f000f0444007a
:1083f40089f62f008f844400caf32f000f0545002f
:108404004bf52f008f8545000d00e0000c00320075
:108414004201dd00080241008001400063807c00cd
:10842400cf80de00008abe000a01410063807d0027
:10843400cf80de000089be006163b9000f00370001
:108444004201dd00880141000002400064807c009c
:10845400cf80de0093094000d39148000a01410017
:1084640064807d00cf80de001209400052914800f4
:108474006160b90006034000878348008502e80074
:10848400e28f520002003c0005007800deff370056
:10849400869f8800979f8800e5878800e633ef0071
:1084a4007fb097000000e900f0b79f009cff3a00fe
:1084b400e08788000605be0081f42f008f8040000d
:1084c400e1b79f00cef32f000f0747004d30210086
:1084d400000678004200dd0062dd2f000f0141003c
:1084e4000204400043db2f008f81410000804100e3
:1084f400f0389100603891004209dd00ce00de00c2
:10850400810071004200dd00c25d200003002000f4
:108514002be10700ce09dd00c200de00818071007e
:108524004e00dd00008cbe001e00be00c25d2000b7
:108534000300200022e107000004be006fb1970091
:1085440032001400a2801c000004be00009fbe0084
:10855400c25d2000030020000a00be0018e10700ed
:108564000005be00c949dd00c744de0089847100ee
:108574004944dd009d0e4400dd964c000c06e800e5
:108584006fb0970064004000e0b79f00f08646009b
:10859400e20f560002003c000c007800cdff3700cb
:1085a4008a9f88009b9f8800ec8788001100200028
:1085b40081bf9f004df72f008f86460066874600d7
:1085c400e613e200feff3200de73ec00029f80003f
:1085d400139f800061014100e0814900029f8800ef
:1085e400139f880040c0b3001e0a0700f2f0b700d2
:1085f40050c0b3001b0a0700f3f0b70060c0b3001b
:10860400180a0700f4f0b70070c0b300150a070099
:10861400f5f0b70080c0b300120a0700f0f0b7000d
:1086240090c0b3000f0a0700f1f0b7000040eb0060
:108634000c0a0700f8f0b700210f210091407800e0
:108644008180fb00f3d0bf004800dd0000804000c3
:10865400a09f9d00410f2100914078008180fb0084
:10866400f5d0bf004800dd0080804000b19f9d0030
:10867400010f2100914078008180fb00f1d0bf0000
:108684004800dd0080804000c19f9d0089002000db
:108694000004eb00a3db2f008f8541002ade2f00ae
:1086a4000f054500ac3e210009007800ec0a0700e4
:1086b400ea007c0001005000e8007e00811d5000ab
:1086c4008904e8000884e800eb8f5400f6ff3a00c0
:1086d40040db2f000f00400070014000ee0040001e
:1086e40000dc2f000f0040002007070039060700b8
:1086f400fe53e200130032002040210041c1b300c8
:1087040090cf100003003a0011c0b300014078007c
:10871400120307000254ed0002f4b7004240a9001e
:1087240002003c0040c1b30002f4b70071e207004c
:108734000004e00003003200613f210010c0b300d8
:1087440030030700d662a8008d00780040db2f00bc
:108754000f004000c1f907006c84460088007800cf
:1087640002dc2f000f00410024fb07007281460049
:10877400880078000d00780045fc07008e00780022
:10878400a3db2f000f80410068fa07008e017800f8
:108794000001eb0044f52f000f02420068dd2f00ba
:1087a4000f04440002004100080040001000be0015
:1087b4004088de00cf80de003300100000327900f4
:1087c4000281e800e60f5100f6ff3a0089f92f0014
:1087d4008f844400b09f8000010020004a09dd001e
:1087e400c600de00810071004a00dd004206200060
:1087f4000300200081e00700908f9f0060a08000ac
:1088040089007800b7fd070040a0800051a08000d7
:108814008ae007000001be00a1f92f008f8040000c
:1088240002007800b7fd07008802780063dc2f009f
:108834000f82410083de2f008f8141007881460042
:108844008d00780066804600acf507001f8897000d
:1088540043f22f008f8141000d01780099007800c8
:10886400d0f807005f109700a08f9f00bf109700fb
:10887400b18f9f00d662a9000fb997000200e000f3
:108884003700320048fa2f000f044400820420000d
:108894008000eb00080078001cdf07000801780066
:1088a40031002000e00f21000f0907006c01440093
:1088b40031002000c01021000b090700780144009a
:1088c40031002000a01121000709070082fc2f00bd
:1088d4000f0141003100200080122100020907002d
:1088e40042fd2f000f0141003100200060132100e0
:1088f400fd08070002fe2f000f01410011002000b7
:1089040040142100f80807007c845700080178000f
:1089140011002000a0142100f308070082f62f00a4
:108924000f01410038197800281178000fa897002a
:108934009fa89700e0379f00f1379f006f90970042
:10894400ff909700803f9f00913f9f0031002000df
:1089540000152100e40807008000eb0081bf9f00a0
:1089640042db2f000f01410091002000e01521009f
:108974001d0907002220210081002000201721006a
:108984002c0907007881460031002000e0172100ff
:10899400150907007281460031002000601821008b
:1089a400110907000d01780031002000e0182100b2
:1089b4000d09070042f52f000f014100310020008e
:1089c40060192100080907006c814600310020006d
:1089d400e0192100040907000901780011002000b2
:1089e400601a2100000907007e8146003100200042
:1089f400a01a2100fc080700a2f52f000f01410076
:108a04009f899700030978004f289700e02f9f0063
:108a1400af889700f12f9f0031002000201b210018
:108a2400f108070063dc2f000f81410041002000a2
:108a3400a01b2100cf08070062dd2f000f014100b9
:108a440031002000c01c2100ca0807000004eb000c
:108a540088379f00509f800090379f00619f80005f
:108a6400a1379f00729f8000b2379f0002f62f004b
:108a74000f01410041002000a01d2100da08070079
:108a8400389f8800ca22a800cdfe3700801f7800d6
:108a94008460a90010002000309f88004f007800f7
:108aa40000400600809fbe008580a900e10e2100e1
:108ab40091407800edd0bf008180fb000080fb0076
:108ac4000000e900808f50000a003d0010002000e3
:108ad400e09e8800ee70ec00eed0bf000080fb004a
:108ae4005102210060c078000080fb002011880042
:108af40001003700dc33ef004f00be0000400600e9
:108b04003600f800809fbe00829fbe00849fbe0096
:108b1400869fbe00881f78008560a9001800200089
:108b240017003700801f780023d0bf0022f0b70061
:108b34004f007800801f780024d0bf0023f0b700d6
:108b44004f00780003e2070024f0b700220221005e
:108b540012417800310221009140780081404100a7
:108b640000c04000f24f410005003a00e10221003c
:108b7400914078000104e10001003a000881880076
:108b840022c2bf000008a300e6ff3a004f047800a9
:108b94004f03be004f02be004f01be004f00be0097
:108ba4003600f9000040060087e0a90000400600f6
:108bb40087c0a900004006003400f800881f780030
:108bc40008c0b300a80188004f0478008020a900e1
:108bd4000000fe003400f900004006003400f800f4
:108be400881f780008c0b300a80188004f047800eb
:108bf4008060a9000000fe003400f9000040060077
:108c04003400f800881f780008c0b300a801880069
:108c14004f0478008040a9000000fe003400f900f1
:108c2400004006003400f800881f780008c0b30034
:108c3400a80188004f0478008080a9000000fe008d
:088c44003400f90000400600b5
:020000040000fa
:108c4c00881f780000047800a0022700d1f82300c8
:108c5c00a9de0700008cbe00a0022700d1f823007b
:108c6c00a7de0700200498003104980000002000c3
:108c7c00010024004004980051049800d0cc2c0032
:108c8c00c1dc23006004980071049800d0cc2c0047
:108c9c00c1ec2300200c9800310c9800000020003f
:108cac0001f82300400c9800510c9800600c9800bf
:108cbc00710c980070712b0011b52300000c9800fa
:108ccc00110c980050582000b19a23000014980001
:108cdc0011149800e0102400a17e230020149800a9
:108cec003114980070862f0041af2b00401498006f
:108cfc0051149800c05a2c0071aa230060149800db
:108d0c00711498004f04780000000600ccff070097
:108d1c00000006003800fa00889fbe008a9fbe0043
:108d2c008c9fbe0000057800c0fb2f000f00400098
:108d3c00c3ff070002e02f00f36f24006f98970029
:108d4c00ff98970038de07000004be006011b800e1
:108d5c006dde07000000e00003003500000020007d
:108d6c0001f02300020037000000200001f02b006e
:108d7c000801be0067de0700c3de0700008dbe00e1
:108d8c0002e02f00f36f24000fa097009fa0970024
:108d9c0025de07000004be006011b8005ade070093
:108dac000000e000030035000000200001f023006b
:108dbc00020037000000200001f02b000801be006b
:108dcc0054de0700b0de070020059800310598003e
:108ddc0002002000032024002fa09700bfa09700c2
:108dec0011de07000004be006011b80046de07006b
:108dfc000000e000030035000000200001f023001b
:108e0c00020037000000200001f02b000801be001a
:108e1c0040de07009cde07004005980051059800d5
:108e2c0002002000032024004fa09700dfa0970031
:108e3c00fddd07000004be006011b80032de070043
:108e4c000000e000030035000000200001f02300ca
:108e5c00020037000000200001f02b000801be00ca
:108e6c002cde070088de070060059800710598006d
:108e7c0002002000034824000fa897009fa8970029
:108e8c00e9dd07000004be006011b8001ede07001b
:108e9c000000e000030035000000200001f023007a
:108eac00020037000000200001f02b000801be007a
:108ebc0018de070074de0700000d9800110d9800f5
:108ecc0002e02f00f36f24002fa89700bfa8970093
:108edc00d5dd0700020020004333240090dd07009d
:108eec000001be00d0dd0700020020000322240098
:108efc00cddd07000200200003c02300cadd0700ff
:108f0c000004be006011b800ffdd07000000e000a7
:108f1c00030035000000200001f0230002003700a0
:108f2c000000200001f02b000801be00f9dd070055
:108f3c0055de0700200d9800310d98006fa19700a9
:108f4c00ffa19700000020000120240074dd070021
:108f5c000004be006011b800ebdd07000000e0006b
:108f6c00030035000000200001f023000200370050
:108f7c000000200001f02b000801be00e5dd070019
:108f8c0041de07002015980031159800325c2f0047
:108f9c00c31124002fa09700bfa0970060dd07002d
:108fac000200200003f023009fdd07006fa1970053
:108fbc00ffa197009cdd07000200200003b82400ed
:108fcc0099dd07000004be006011b800cedd07007b
:108fdc000000e000030035000000200001f0230039
:108fec00020037000000200001f02b000801be0039
:108ffc00c8dd070024de0700400d9800510d9800d5
:10900c00b2fd200093fc23006fa09700ffa09700f7
:10901c0085dd07000200200003b8240082dd070074
:10902c000004be006011b800b7dd07000000e000ce
:10903c00030035000000200001f02300020037007f
:10904c000000200001f02b000801be00b1dd07007c
:10905c000dde0700600d9800710d980002e02f00e6
:10906c00f36f24004fa09700dfa097006edd070080
:10907c00e2d52800631f240029dd07006fa19700ab
:10908c00ffa1970068dd0700020020000378240090
:10909c0065dd07000004be006011b8009add070012
:1090ac000000e000030035000000200001f0230068
:1090bc00020037000000200001f02b000801be0068
:1090cc0094dd0700f0dd07000015980011159800dd
:1090dc00c10220008a8040000000eb006011b80043
:1090ec008298be000000e800e30f5000fcff3a003d
:1090fc00cd0320008a8646000006eb006fa0970087
:10910c00ffa09700e0b79f00f1b79f000fa8970052
:10911c009fa8970080bf9f0091bf9f006160b9001e
:10912c00fadd07000c00e00003003d000200200007
:10913c000378240077dd07000200200003f02300f1
:10914c0074dd0700020020000322240036dd070036
:10915c000200200003c0230033dd07000004be0022
:10916c000200200003c824006fb09700ffb09700e6
:10917c002ddd07000fb997009fb997002add070076
:10918c000005be000801be000800be0026dd070079
:10919c000200200003f823005edd07000001be0082
:1091ac000a00be00dedc07000004be006011b8003f
:1091bc0055dd07000000e000030035000000200032
:1091cc0001f02300020037000000200001f02b000a
:1091dc000801be004fdd0700abdd0700801e7800e4
:1091ec000c06e80000082000800f5600cbff3a0068
:1091fc004f06be004f05be004f04be000080fa00b3
:10920c0000000600000278006000b800f50720009e
:10921c00850f5100e08f590004003e000200410010
:10922c00c003b00060007a000100200000000600be
:020000040000fa
:10923c0023c2bf000008a300fdff32002342a80098
:10924c002362a800f00f2000201188000000060007
:10925c000600fa00f04f500014003e00a0ff9f00e3
:10926c00b1ff9f000040eb00c0ff9f0036df0700fe
:10927c000004e000fdff3a00edff07006680570098
:10928c00f8df070030df07000004e000fdff3a00c4
:10929c0082382100e68057004000200099df07004b
:1092ac00110020000000e000010032008000eb0003
:1092bc00010078000080fa00000006008180fb00ad
:1092cc008100e900cf08de002146b000e0ff070076
:1092dc000080fb00000006000001780041c6b300ce
:1092ec0000b02400800f5100050032008000eb001c
:1092fc0000602900800f510004003a0051c6b300f1
:10930c000040eb00d2ff07008080fb0001007800da
:10931c000000060001c6b300cdff07000080fb0073
:10932c0000000600f00f20001ae0070007e007001d
:10933c000041eb00f10f2000810f500001003200c2
:10934c0012c0b300024078000004a2000080fb00b1
:10935c00000006008180fb008100e900cf08de00e0
:10936c0042c5b30081405100b9ff07000080fb00eb
:10937c00000006008001780081a0800092a080008f
:10938c00828f50000200310002007800020037008a
:10939c000100780082007800830f5000050039002e
:1093ac00818f51000200310001007800010037006c
:1093bc000300780082a0880093a0880000000600bb
:1093cc00810f500005003600820f50000a00390052
:1093dc00828f50000500390006003700820f5000c4
:1093ec0005003e00828f500002003600020078001b
:1093fc000100370001007800000006000200fa00ae
:10940c00881f78000104780038df07000004e000b2
:10941c000e00320002712200e48057002000200070
:10942c0038df07000000e00008003a004ff8970012
:10943c008080fb00c808dd005ff897000080fb000f
:10944c00008c400010002000010037000000eb00f1
:10945c004f0478000080fa00000006008180fb00b9
:10946c008100e900cf08de0012c5b3008140510035
:10947c0077ff07000080fb00000006000200fa00e6
:10948c00881f780001047800e1c5b30070ff070065
:10949c000004e0000e00320002712200e48057004c
:1094ac002000200017df07000000e00008003a0051
:1094bc004ff897008080fb00c808dd005ff897002c
:1094cc000080fb00008c40001000200001003700e1
:1094dc000000eb004f0478000080fa00000006004a
:1094ec000600fa00889fbe008a9fbe0000457800e7
:1094fc00814578000000eb00f0cf50004d003e009d
:10950c00aaf79f0000cab300b0f79f000040eb0021
:10951c00c0f79f008cde07000004e000fdff3a005e
:10952c0043ff0700ee845700090078004ddf070069
:10953c0085de0700004478000004e000fcff3a00e0
:10954c00823821008900780040002000edde070001
:10955c002362a900aaf79f00a0cab300b0f79f002e
:10956c00c8f79f0078de07000004e000fdff3a001a
:10957c002fff0700090078003adf070072de0700b2
:10958c00004478000004e000fcff3a00823821001f
:10959c008900780040002000dade07002362a90071
:1095ac00aaf79f0050cab300b0f79f00c8f79f00fe
:1095bc0065de07000004e000fdff3a001cff070019
:1095cc000900780027df07005fde07000044780001
:1095dc000004e000fcff3a0082382100890078008a
:1095ec0040002000c7de07002362a900aaf79f00f5
:1095fc00bbf79f00c8f79f0053de07000004e00094
:10960c00fdff3a000aff07000900780015df07008c
:10961c004dde07000004e000fdff3a008238210017
:10962c008900780040002000b6de07002362a90004
:10963c00100020004f05be004f04be000080fa0051
:04964c000000060014
:020000040000fa
:1096500016c2bf000008a300fdff3a0016c2bf00fb
:109660000028a300faff3a0016c2bf000038a3008a
:10967000f7ff3a0016c2bf000048a300f4ff3a000b
:1096800019c2bf000068a300f1ff3a000000060005
:1096900017e2a90017a2a9001782a8001762a90063
:1096a0001742a9001722a8001702a90016e2a90074
:1096b00016c2a90016a2a9001682a9001662a90066
:1096c0001642a9001622a9001602a9007001200066
:1096d000a0108800bdc0bf0081cfb3000140600072
:1096e0000024a000bde0b70018c2a9009a20a9007c
:1096f00017e2a800006a2800110020002b070700cd
:10970000100020000000060017e2a9008a40a9000e
:109710008a20a9009a20a900803e20000100200094
:1097200061005000e0805800fdff3a00d8ff0700bc
:1097300005000700006a2800110020001b07070031
:1097400010002000000006008a40a9009a40a800ee
:10975000006a2800110020001407070010002000f4
:10976000000006008a40a9009a40a90010002000cd
:109770000000060016c2bf000008a300fdff3a006b
:1097800016c2bf000028a300faff3a0016c2bf00ad
:109790000038a300f7ff3a0016c2bf000048a3003c
:1097a000f4ff3a0016c2bf000018a300f1ff3a0010
:1097b00010c0b3001ef4b7001602a800007122000a
:1097c000010020001e54e20002003a0010002000b8
:1097d0000400370061005000e0805800f9ff3a00b3
:1097e0000000eb000000060060c0b3001ef4b700ec
:1097f00018c2bf000038a3000a0032001622a800d9
:1098000000712200010020001e54e20002003a0014
:10981000100020000400370061005000e080580074
:10982000f9ff3a000000eb000000060030c0b30072
:109830001ef4b70016c2bf000008a30017003a00cc
:1098400016c2bf000028a30014003a0016c2bf00d1
:109850000038a30011003a0016c2bf000048a30060
:109860000e003a0016c2bf000018a3000b003a0019
:1098700016a2a9001682a800007122000100200093
:109880001e54e20002003a001000200004003700dd
:1098900061005000e0805800f9ff3a000000eb0042
:1098a0000000060030c0b3001ef4b70016c2bf00af
:1098b0000008a30017003a0016c2bf000028a3004a
:1098c00014003a0016c2bf000038a30011003a008d
:1098d00016c2bf000048a3000e003a0016c2bf0027
:1098e0000018a3000b003a0016a2a8001682a800d8
:1098f00000712200010020001e54e20002003a0024
:10990000100020000400370061005000e080580083
:10991000f9ff3a000000eb000000060000027800aa
:1099200040c0b3001ef4b700027122000300200003
:1099300016c2bf000008a3000c003a0016c2bf0008
:109940000028a30009003a0016c2bf000038a30097
:1099500006003a0016c2bf000048a30003003a0008
:1099600019c2bf000068a300080032006101510065
:10997000e08159000d003200edff370080108000bb
:10998000004a780010002000090037001662a80085
:10999000006a2800110020001e54e200f7ff320088
:1099a00061005000e0805800fbff3a000000eb002f
:1099b0000000060050c0b3001ef4b7001642a80015
:1099c00000712200010020001e54e20002003a0053
:1099d000100020000400370061005000e0805800b3
:1099e000f9ff3a000000eb000000060021c0b300c0
:1099f0008000fd001ef4b7008000fd000000fb00a9
:109a0000901088001602a8000071220001002000ba
:109a10001e54e20002003a0010002000040037004b
:109a200061005000e0805800f9ff3a000000eb00b0
:109a3000000006008a40a9001e74ef0000400600e6
:020000040000fa
:109a4000cf80de000004b0000180b0004909dd00d5
:109a50004700de0000007100c788de000010b00083
:109a6000f01fb20080004000c0202a006100780092
:109a700000000600cf80de000004b0000180b000ce
:109a80004909dd004700de0000007100c788de00e4
:109a90000010b000f01fb20080004000c0e02900bc
:109aa0006100780000000600f10f2000810f5000d7
:109ab00005003e00010060000000400061e0280059
:109ac0006080780000000600010020000008b0005f
:109ad0000180b0004809dd004800de000000710090
:109ae000c888de00000040006200290060007900a4
:109af00000000600cf80de000002b0000180b00050
:109b00004a09dd004600de0000007100c688de0064
:109b1000800040000040200080804000802029001c
:109b20006100780000000600f2032000130020000e
:109b30000100e00003003a000001be000204b00092
:109b40000380b000491add004710de0000007200fb
:109b5000c718de000000400042a028006000790025
:109b600000000600010020000004b0000180b000e9
:109b70004909dd004700de0000007100c788de00f3
:109b80008000400040a0280061007800000006002e
:109b90008000780002002200f0ff2700808f500034
:109ba0000f00320002002e0010002800808f5000ad
:109bb0000b0032006108b9000004b0000180b00061
:109bc0004909dd004700de0000007100c788de00a3
:109bd000000040000020b000a2a029006001790030
:109be0000200780000000600889fbe000001780097
:109bf0000000e00001003d000001ea006114b9002e
:109c0000010278000100e00001003d000102ea00cd
:109c10006123b9006102b9006109b9000100e000e7
:109c200002003a000000e0002f003200860f5400ce
:109c3000878f5c0015003c000100e0000700350044
:109c40004f28dd00c120de00810070004f20dd00c4
:109c50005cdb0700ceff0700230037004f28dd0044
:109c6000c120de00810070004f20dd006000100088
:109c7000e08018000601be0052db0700c4ff0700a9
:109c8000f1ff270001004000170037000000e0004e
:109c90000c0034004f18dd00c110de0081007000a0
:109ca0004f10dd0060001000e08018000401be00cd
:109cb00044db0700b6ff0700f1ff2300010040006e
:109cc000090037004f18dd00c110de008100700070
:109cd0004f10dd000801be003adb0700acff0700b3
:109ce00011002c00010040004f04be0000000600df
:109cf000889fbe000003be000002be00e00f5000bf
:109d0000e08f580002003d0060021000e082180061
:109d10000204be00e00f5100e08f590002003d0038
:109d200060041100e0841900e00f5100e08f590039
:109d300004003a000000eb00e00f5300e08f5b00ee
:109d400031003200880f5200898f5a0016003c0003
:109d5000e00f5100e08f5900070035004f38dd005b
:109d6000c130de00810070004f30dd0015db0700e0
:109d700087ff0700240037004f38dd00c130de00c8
:109d8000810070004f30dd0060001000e08018009e
:109d90000801be000bdb07007dff0700f1ff270075
:109da0000100400018003700e00f5300e08f5b0017
:109db0000c0034004f18dd00c110de00810070007f
:109dc0004f10dd0060001000e08018000601be00aa
:109dd000fcda07006eff0700f1ff230001004000de
:109de000090037004f18dd00c110de00810070004f
:109df0004f10dd000401be00f2da070064ff070027
:109e000011002c00010040004f04be0000000600bd
:020000040000fa
:109e1000881f780000122a007100200063050700e7
:109e20000044eb000844e800006a2800110020000c
:109e30005e05070071c0b30020c2b30071010700c6
:109e40000008a3000a003200f44f5400f5ff3a0066
:109e5000a8c0b300f1c7b30020c2b3006901070076
:109e6000a1002000e14f500009003a000200370035
:109e700018c0b300f7ff3700a2c0b30031c0b30071
:109e800020c2b300b3010700084060008000fb005f
:109e9000010078004f04780000000600881f780059
:109ea00000482800e1012000400507000041eb00c8
:109eb00031c0b30020c2b300a60107006a446000ad
:109ec00000122a007100200038050700a2c0b3006c
:109ed00031c0b30020c2b3009e01070000406400ff
:109ee0000000fb004f047800000006000400fa00a8
:109ef000881f7800d5c2bf00a10020000008a30081
:109f00003100320023c0b30012c8b300e68057000e
:109f100020c2b3005c0107002ff897000084fb000b
:109f20004844dd003ff897000080fb000004740007
:109f30006140b90078da07000800e00003003d0046
:109f40000200200003782400f5d9070040a0880013
:109f500051a08800f1c7b30020c2b3002901070057
:109f6000e68057008058780023c0b30002c8b300d1
:109f700020c2b300440107002ff997004811dd000b
:109f8000030020003ff897000080fb000100200044
:109f90000001710081817100c819dd000280fd009f
:109fa000824178000041eb004ff897000080fb00f1
:109fb00001002000000171008181710062a0880011
:109fc00073a0880011002000010078004f04780081
:109fd0000080fa00000006000400fa00d5c2bf00ad
:109fe000a10020000008a30021003200f1c7b30047
:109ff00020c2b30003010700e480570080587800b6
:10a0000023c0b30002c8b30020c2b3001e01070082
:10a010004ff897004800dd00010020005ff997002d
:10a020000281fb00030020000200700083807000aa
:10a03000c808dd000080fd00804078000040eb0093
:10a040006ff997000281fb000300200002007000fe
:10a05000838070004c09dd004400de0000007100c8
:10a06000c488de0060a0880071a088001100200074
:10a07000010078000080fa000000060080407800af
:10a0800020c2b300df0007000000fb000000060054
:10a09000014178008040780020c2b3002d01070004
:10a0a0000000fb0000000600889fbe008a1f7800a9
:10a0b000004178008104780021c0b30020c2b300c1
:10a0c000240107006145600012c0b30031c0b30035
:10a0d00020c2b3001f01070000447800006a280076
:10a0e00011002000b104070011c8b30020c2b30062
:10a0f000c4000700804c7800084065000000fb00a9
:10a100004f0578004f04be0000000600889fbe0087
:10a11000004178000144780021c0b30020c2b300a0
:10a120000c010700e14460000841780011c0b30051
:10a1300020c2b3000701070080c4640022c0b3003e
:10a1400031c0b30020c2b300020107000044780010
:10a1500000122a00710020009404070008c0640067
:0ca160000000fb004f04be0000000600e1
:020000040000fa
:10a16c00881f780022c0b30082407800c0c3b300bf
:10a17c00f50007006144600082c1b3008040eb0031
:10a18c00c0c3b300f00007000044640002c2b30077
:10a19c0011c0b300c0c3b300eb000700004464005f
:10a1ac000041eb0021c0b300c0c3b300e6000700c0
:10a1bc00004064000000fb004f0478000000060023
:10a1cc0080407800c0c3b3008b0007000000fb0088
:10a1dc00000006000141780080407800c0c3b30045
:10a1ec00d90007000000fb0000000600889fbe009d
:10a1fc000004780031c0b300c0c3b3007e00070078
:10a20c00c804dd0041c0b300c0c3b3007a0007002e
:10a21c000080fb0000807400cf80de00bbd90700fb
:10a22c00008cbe00100020004f04be000000060091
:10a23c00889fbe000004780051c0b300c0c3b300b7
:10a24c006d000700c804dd0061c0b300c0c3b300db
:10a25c00690007000080fb0000807400cf80de00e6
:10a26c00aad90700008cbe00100020004f04be00cd
:10a27c0000000600889fbe000004780071c0b30087
:10a28c00c0c3b3005c000700c804dd0081c0b3008c
:10a29c00c0c3b300580007000080fb0000807400ae
:10a2ac00cf80de0099d90700008cbe001000200082
:10a2bc004f04be00000006000c00fa00889fbe0090
:10a2cc008a9fbe000004be0002057800d5c2bf0004
:10a2dc00a10020000038a3001d00320063c0b300b1
:10a2ec0032c0b300ee805700c0c3b3006300070058
:10a2fc00e14560006d815700f4815700678257007b
:10a30c0072f897004800dd009280fb008119700004
:10a31c000281e800820f5200f9ff3a006fb09700fb
:10a32c00cf80de0079d90700008cbe007fb097008b
:10a33c00cf80de0075d90700808cbe000fb8970067
:10a34c00cf80de0071d90700008dbe008b00fb00b2
:10a35c00010078004f05be004f04be000080fa00db
:10a36c00000006000c00fa00889fbe008a1f7800cf
:10a37c000004be0002057800d5c2bf00a100200079
:10a38c000038a3001700320063c0b30032c0b30022
:10a39c00ec805700c0c3b30038000700e1426000f6
:10a3ac006b815700f28157006582570072f8970055
:10a3bc004800dd009280fb00811970000281e800ea
:10a3cc00820f5200f9ff3a007fb09700000c780022
:10a3dc000fb89700800c78001fb89700000d78001c
:10a3ec008500fb00010078004f0578004f04be008b
:08a3fc000080fa0000000600d9
:020000040000fa
:10a404000200fa00889fbe008a9fbe0000457800c3
:10a414008145780001003700bafc0700d4fc07002e
:10a42400614460000a4078006ffd07000044640046
:10a434000b4078006cfd070000446400e9fc070051
:10a44400004464000a40e80067fd0700804464009b
:10a454006a80570030fd07000044780010fd0700b3
:10a4640053fd070008c06400ebff3200eff09700d3
:10a474000100fb004f05be004f04be000080fa003f
:10a4840000000600889fbe008a9fbe008c1f7800d3
:10a4940000447800010678008244780083457800ff
:10a4a400b3fc070061456000084078004efd0700da
:10a4b40000456500094078004bfd070080446500b5
:10a4c400c8fc070080c464000844e8000840780021
:10a4d40045fd070000c564000b04e00016003200cf
:10a4e4000c0478008b4478000b40e9000080fb00ea
:10a4f400000046008005e8000800780006fd07001b
:10a504000a4560000804e8008944e90003003a00b1
:10a51400e3fc07000045650002003700c2fc0700a9
:10a524000045650016c2bf000048a300fdff3a00c5
:10a53400888f5500f0ff3a001dfd07000a00fb005c
:10a544004f0678004f05be004f04be000000060011
:10a55400889fbe008a9fbe00804578000145780030
:10a56400824478000100370066fc070080fc070085
:10a57400614460000b4078001bfd07000044640048
:10a584000a40780018fd0700004464000940780080
:10a5940015fd07000044640005fd07000040640049
:10a5a400f1ff32000000fb004f05be004f04be0067
:10a5b400000006000200fa00881f78000040eb004b
:10a5c400c0ff9f006afc07006144600000c1b30043
:10a5d40005fd07000044640010c0b30002fd07003d
:10a5e400004464007ffc07000044640010c1b30011
:10a5f400fdfc07000044640064805700c6fc0700ab
:10a6040000446400a6fc070000446400e8fc070062
:10a6140000406400ebff3200cff897000100fb001c
:10a624004f0478000080fa0000000600881f7800bc
:10a634004ffc07006144600000c1b300eafc07005e
:10a64400004464000040eb00e7fc070000446400a1
:10a6540050c0b300e4fc070000446400d4fc0700cd
:10a6640000406400f2ff32004f047800000006004e
:10a6740006fc07000000060032fc0700000006008c
:08a6840037fc0700000006008e
:020000040000fa
:10a68c001c1400000200000002000000000000008a
:10a69c00fe1000000401000000000000dc130000ac
:10a6ac002c00000002000000000000000000000070
:10a6bc00000000000000000000000000000000008e
:10a6cc00000000000000000000000000000000007e
:10a6dc00000000000001000000001400141414001d
:10a6ec000300000050080000ae080000000000004d
:10a6fc001e140000020000000000000008140000fe
:10a70c000800000000000000f8120000e400000047
:10a71c000000000010140000080000000000000001
:10a72c0018140000040000000000000002120000d9
:10a73c00f6000000020000004358300030323300b5
:10a74c0000006f009a9f3a005561e70036e58000e3
:10a75c0014b7a900808c3d008c477d00365f1e002d
:10a76c00a0ba0b008bdf3700dc2049003e384d00cf
:10a77c00eab74a00d98bb700ba0ca000bab497005c
:10a78c00c03d0000000000000000000000000000c0
:10a79c000000000000803f00de9dd800bea2bb0080
:10a7ac00e0ba6b007e8ebc0000ed1900c12ffa00e0
:10a7bc0038bbfe00ccd23e00b3674e003a15bb004e
:10a7cc003e3f9400e0b03b00ccf012003cc9f800d6
:10a7dc004d3ea00073173e0000000000000000007a
:10a7ec000000000000000000000080003f0100009d
:10a7fc00000080003f00000000000000000000008e
:10a80c0000000000000000000000000000803f007d
:10a81c00000000000000000000000000000000002c
:10a82c000000000000000000803f0000000000005d
:10a83c00000000000000000000000000000000000c
:10a84c00000080003fe3250093c23f00c6f2c00029
:10a85c00c3352b004300000080bf0400e78c3b0095
:10a86c00789c6200be18b4001039000000803f00d4
:10a87c000000000000000000803f0000000000000d
:10a88c002014000002000000000000000000000086
:020000040000fa
:10a89c00fe51a90007e2a90080002000501088009a
:10a8ac0007a2a8000782a8000762a9000742a90016
:10a8bc000722a8000702a90006e2a90006c2a90007
:10a8cc0006a2a9000682a9000662a9000642a900f8
:10a8dc000622a9000602a90008c2a9008600a90048
:10a8ec008620a900acc0bf0081cfb300014060003e
:10a8fc005040b300ace0b700acc0bf00f1c8b3002f
:10a90c00014060000044a000ace0b7009620a90014
:10a91c00e00f210000908800fe11a900fe31a90073
:10a92c00fe51a90007e2a800803e20000000e900cb
:10a93c00feff3a009600a800803821000000e900d4
:10a94c00feff3a0000000600809fbe003400f800b5
:10a95c0000c0b300a001880008c2bf000028a300fb
:10a96c002900320008c2bf000058a30026003a009c
:10a97c00fe51ab0010003a000010800000908000e7
:10a98c00904078008000fd001cf4b7008000fd00b2
:10a99c001080fb00101088000782a80008c2bf00be
:10a9ac000008a300fdff3a000140e9001cf4b700c9
:10a9bc00fe51a80034003700c141210091407800bd
:10a9cc000104e0000c003400001080000012ec00c8
:10a9dc00009088001080fb00101088000782a800ef
:10a9ec0008c2bf000008a300fdff3a000140e900c7
:10a9fc001cf4b70024003700e00f21000090880001
:10aa0c00fe51a9002000370008c2bf000028a30097
:10aa1c0006003a0008c2bf000058a30003003a0029
:10aa2c0000108000fe11a8001700370008c2bf00fc
:10aa3c000028a30014003a0008c2bf000058a3006d
:10aa4c0011003200fed1bf000008a3000500320047
:10aa5c00fe11a900fe31a800001080000032b400e5
:10aa6c00090037000018a300070032000010800016
:10aa7c000190800080487800fe11a900fe31a900e9
:10aa8c00e00f2100009088008600a9003400f90036
:08aa9c004f00be00004006005f
:020000040000fa
:10aaa400a9c0bf0081cfb300014060000024a00012
:10aab400a9e0b700aac0bf00f1c8b300014060001c
:10aac4000045b300aae0b70000000600d662a80063
:10aad40010242400f100200061005000e0805800a0
:10aae400fdff3a00d662a90000242400f1002000f2
:10aaf4000081eb008081eb0061005000e080580091
:10ab0400820f5000838f5800fbff3a0000000600bc
:10ab1400800078001080fb004800dd009140900028
:10ab24008100fb0002f02f008280600001004000e1
:10ab340000000600800078001080fb004800dd0063
:10ab4400914090008180fb0001004000000006005d
:10ab54000400fa00c3ff9f00d2ff9f00e1ff9f00a3
:10ab6400f0ff9f006fb89700ffb897000080fa00cd
:10ab7400000006000200fa00e0ff9f00f1ff9f00c2
:10ab84007fb897000080fa00000006000080fb00f8
:10ab9400000006004800de00000006000200fa0083
:10aba400f0bf9f00eff897000180fb000080fa00df
:10abb400000006000200fa00f0bf9f007ff8970033
:10abc4000080fb000080fa00000006000400fa0088
:10abd400e0bf9f00f1bf9f00cff897000180fb000a
:10abe4000080fa00000006000400fa00e0bf9f00a5
:10abf400f1bf9f005ff897000080fb000080fa001f
:10ac0400000006000400fa00e0bf9f00f1bf9f00af
:10ac14006ff897000080fb000080fa000000060037
:10ac24000400fa00e0bf9f00f1bf9f007ff8970087
:10ac34000080fb000080fa0000000600b2fd200046
:10ac44009304240038d60700020020004333240074
:10ac540077d6070000000600b2fd2000930424000c
:10ac640073d6070002002000433324002ed60700c9
:10ac7400000006000000e000090034008001eb0041
:10ac8400f22921008000eb008100e800828f50004f
:10ac9400fdff3a008301e800830f5000f9ff3a00fa
:04aca40000000600a6
:020000040000fa
:10aca800800078001080fb008001e9000042eb0082
:10acb80012002000828f5100070036000042eb008e
:10acc8001200200062c07800004242000201e80041
:10acd800830f5100fbff3a000440ea0000f17800be
:10ace80000000600889fbe008a9fbe008c1f780067
:10acf80000067800010578004208dd000c047800a1
:10ad080000dce8000100e000120032008204780054
:10ad18008005eb001900be00abff0700004c78006f
:10ad28001900be00afff0700104498001900be00cc
:10ad3800b3ff0700204498003900be00b7ff0700a2
:10ad480030449800640444008b05e8008b0f5500dc
:10ad5800f0ff3a000c007800d1ff07000000eb007c
:10ad68004f0678004f05be004f04be0000000600e5
:10ad780000037800810278004208dd00860178002f
:10ad880080d9e8000100e000120032000002eb0068
:10ad9800924978001200be00c80bdd004800de00b2
:10ada80000807300c888de0090419800224090001f
:10adb800a04198003200be004888de00cf80de0047
:10adc800b0419800e48141000402e800848f5200f9
:10add800efff3a0006007800b1ff07000000eb0023
:10ade800000006008002780001804000850178009c
:10adf80080d9e8000100e000090032000002eb0001
:10ae080092497800320078004880de00904198002e
:10ae18008381e8000402e800848f5000f8ff3a00bc
:10ae2800050078009eff07000000eb000000060008
:10ae38000002780001dae8000100e00005003200b5
:10ae48008001eb0062f279008301e800838f5000f3
:10ae5800fcff3a0092ff07000000eb00000006002c
:020000040000fa
:10ae6800e722a90060c2a90061e2a8006002a90067
:10ae78004a00dd004013880060c2bf000008a3003c
:10ae8800fdff3200401380006002a900e722a800fd
:10ae98000080fb0000000600c842a90060c2a900ab
:10aea80061e2a8006002a9000080fb000008b00071
:10aeb8004800dd004013880060c2bf000008a300fe
:10aec800fdff3200401380006002a900c842a800bc
:10aed8000080fb0000000600c842a90060c2a9006b
:10aee80061e2a8008180fb004800dd00808040000e
:10aef80041138800c01d20000000e900feff3a0051
:10af080040138000c842a80000000600e022a90003
:10af180060c2a90061e2a8006002a9000080fb00ed
:10af28000008b0004800dd004013880060c2bf0080
:10af38000008a300fdff3200401380006002a90052
:10af4800e022a8000080fb000000060080007800d6
:10af5800c842a90040c2a90032002000e50f5000f5
:10af68001d00320009003e0012002000e20f5000d0
:10af78001900320022002000e40f500016003200b1
:10af8800e10f50000f003a00100037005200200077
:10af9800ea0f50001000320003003e00e80f500096
:10afa80008003a000b00370062002000f00f500044
:10afb800090032007200200000022000808f50003b
:10afc80005003200f20f2000030037000001eb00fb
:10afd80001003700420020000200780000e0a000d5
:10afe8004012880000000600c842a90040c2a9001b
:10aff80001102400010070004012880000000600c3
:020000040000fa
:10b00800b0fc2f00301688000000eb0060168800a6
:10b0180090168800c01d2300f0168800f0c3200099
:10b0280020178800000006009460a9009500a80079
:10b038009780a8009a00a8009a80a80095a0a90067
:10b0480097c0a8009540a8000000060005e1a900e7
:10b058000021ef0080382100100888000481a80032
:10b0680004a1a9000421a90004c1a900a580a80081
:10b07800a5a0a900a5c0a9008460a9009460a800a3
:10b0880005e1a8000000060021e3a90021a3a9000a
:10b098002183a8002143a800c0cfb3002163b600d4
:10b0a8007c4050002063b7002063a9002043a9001a
:10b0b8002023a9002003a900f0c1b3002363b60030
:10b0c8002343a9002223a9002203a90025e3a900fc
:10b0d8002563b700f0c3b30024e3b700c0ff2f0017
:10b0e80050198800008c27006019880000000600ad
:10b0f800a4d70700f0f52f00d3d7070032002000af
:10b10800d1f5230000c02c0053d80700000006002a
:10b118008000eb0001138800904320001013880082
:10b1280021138800b4c0bf000044a1000046b3004a
:10b13800b4e0b70061e2a800c842a800c642a9006e
:10b14800e522a900de22a900c842a800e722a8003b
:10b15800e022a800000006000024ef0010002000f4
:10b1680080208800f0e0210090218800000006007f
:020000040000fa
:10b1780081cfb300014078005261b60053a1a90005
:10b1880052e1a900f0c9b3005261b60052c1bf0034
:10b19800014060003040b30052e1b70088e0a900e8
:10b1a800b7c0bf00f1c8b300014060000045b3005c
:10b1b800b7e0b70098e0a80013e1a80013a1a90020
:10b1c80012c1bf00f1ccb300014060000044a000f0
:10b1d80012e1b7001061a9001221a90000000600c1
:10b1e800809fbe0052c1bf0067406000e34f50001f
:10b1f80014003a000a21ef0052c1bf0081cfb3000a
:10b20800014060000014a00052e1b7000a003700b6
:10b21800810a800052c1bf000038a300fcff3a0039
:10b22800c1a0880052c1bf0081cfb30001406000b7
:10b238003040b30052e1b70088e0a9004f00be00db
:10b248000040060052c1bf000038a300f0ff3a00da
:0cb25800f4ff37008500a900004006004c
:020000040000fa
:10b26400ff416000813220009140780002ceb3009b
:10b2740082c0600083c070008000fd0028e3b70036
:10b284008000fd002e23ef00110020008008dd0067
:10b294008119880021e3a8002023a80020c3bf004f
:10b2a4000008a300fdff3200001880002023a9003d
:10b2b40021e3a90000000600ff4160008132200064
:10b2c4009140780002ceb30082c0600083c0700059
:10b2d4008000fd0028e3b7008000fd002e23ef006e
:10b2e400110020008008dd008119880021e3a800f6
:10b2f4002023a8000000060020c3bf000004a20011
:08b3040061006000000006007a
:020000040000fa
:10b30c0019d7070050f42f0023d707009c20a90061
:10b31c006214200001512a0080802a00c9d707003e
:10b32c0000000600f0fd2f001bd70700a201200033
:10b33c000150280080802c00c2d7070000000600b6
:10b34c000fd70700f0fd2f003ed707007205200035
:10b35c00d175290080602c00bed7070000000600c4
:020000040000fa
:10b36c00d662a900d262a900d622a900d222a900d5
:10b37c00c642a800d362a800d302a800d542a900f7
:10b38c00d342a800e442a800e462a800c602a800c8
:10b39c00ca22a900c622a900d282a8000000060079
:020000040000fa
:10b3ac00f03fb1000180b10006003500ee0309004a
:10b3bc0000000000403fb1000180b100fbff3d00e8
:10b3cc001000b000203fb0000200350000800900e2
:08b3dc00000000000000060063
:020000040000fa
:04b3e4000000fe0067
:00000001FF
